:1000000000400020A13E0000E13E0000E33E000071
:1000100000000000000000000000000000000000E0
:10002000000000000000000000000000E53E0000AD
:100030000000000000000000E73E0000E93E000074
:10004000EB3E0000EB3E0000D5460000EB3E00001A
:10005000EB3E000000000000EB3E0000EB3E000025
:10006000EB3E000019410000EB3E0000EB3E0000BB
:10007000EB3E0000EB3E0000EB3E0000EB3E0000DC
:10008000EB3E000079470000EB3E0000EB3E000035
:10009000EB3E0000EB3E0000EB3E0000EB3E0000BC
:1000A000EB3E0000EB3E00000000000000000000FE
:1000B0000000000000000000000000000000000040
:1000C000054B0648033310B51B1A062B03D9044B06
:1000D000002B00D0984710BDD4000020D400002091
:1000E000000000000648074910B5091A8910CB0F17
:1000F0005918491003D0044B002B00D0984710BD6D
:10010000D4000020D40000200000000010B5074CEF
:100110002378002B09D1FFF7D3FF054B002B02D02A
:10012000044800E000BF0123237010BDD40000206C
:1001300000000000586C0000094B10B5002B03D0E4
:100140000849094800E000BF08480368002B02D1B5
:10015000FFF7C8FF10BD064B002BF9D09847F7E713
:1001600000000000D8000020586C0000D0000020E3
:1001700000000000164B002B00D1144B9D4640227E
:1001800092029A1A924600218B460F461348144A4F
:10019000121A04F06AFD0F4B002B00D098470E4B4B
:1001A000002B00D098470020002104000D000D48CE
:1001B000002802D00C4800E000BF04F013FD20002E
:1001C000290004F09FFA04F0E7FCC0460000080094
:1001D000004000200000000000000000D4000020CB
:1001E000EC1E00200000000000000000012303407E
:1001F0000200181E04D1042A03D91068000900E087
:100200000020704710B50400FFF7F0FF0300012045
:10021000002B0BD0013B9B00181DE2181279002A1D
:1002200003D001338342F8D100E0180010BD012251
:10023000016810B5114201D0002903DA102001F045
:1002400093FD03E04910062001F046FE10BD016851
:1002500010B5CB0701D5002903DA102001F084FD89
:1002600006E04910033189100022052001F034FE18
:1002700010BD70B50568AB0728D1042D26D90F2312
:100280002A6846681340062B09D12800FFF7AEFF05
:10029000012383421DDC9A00AE500133F9E7052BA0
:1002A00014D1F30703D4132001F05EFD12E07610A1
:1002B000FF2EF8D82800FFF799FF2C1D230080009F
:1002C0002018984205D91E700133FAE70B2001F07F
:1002D0004BFD002070BD70B50468E30701D4112008
:1002E0002DE04568AB0729D1042D27D90F262B68AF
:1002F00064101E40062E0BD1002C04DD2800FFF7F1
:1003000075FF844201DD122019E0A400605918E055
:10031000331F012B12D82800FFF768FF8000042E3E
:1003200002D12800FFF76EFF002CECDDA042EADBD3
:1003300001232C19E0784000184302E00B2001F063
:1003400013FD70BDF8B5012304681C4201D11120D2
:100350002FE00325466835402AD1042E28D90F23E3
:100360003268641087681340062B0BD1002C04DD23
:100370003000FFF73BFF844201DD122019E0A400AA
:10038000A75113E0052B13D1002CF6DD3000FFF749
:100390002DFF80008442F0DC01231F4201D1132095
:1003A00007E07F10FF2FFAD83419E770280002E029
:1003B0000B2001F0D9FCF8BD006810B5830717D1F8
:1003C000042815D90F2302681340062B02D1FFF72A
:1003D0000DFF0BE0052B05D1FFF708FFC00001233F
:1003E000184308E0042B03D1FFF70CFF4000F6E7A9
:1003F0000B2001F0B9FC10BD10B5032400680440C7
:1004000006D1042804D90F2302681340042B01D01D
:100410000E200CE001F09CFD1022210005F0E2F816
:1004200080239B05C218054B9A4203D9142001F082
:100430009BFC02E001234000184310BDFFFFFF3F7B
:1004400010B501240368234202D04268224203D13E
:100450000D2001F089FC08E004495B1052101B07D5
:100460000A40134318684000204310BDFCFFFF0FF3
:100470000121036810B50B4205D042680A4202D040
:100480008068084203D10D2001F06EFC08E00549A8
:100490005B1052101B070A404010134318600020E5
:1004A00010BDC046FCFFFF0F012303400200181ED1
:1004B00001D0501002E00D22014B1A707047C04667
:1004C000F0000020012303400200181E04D1042A7A
:1004D00003D91068000900E00020704770B50D00D6
:1004E0000400FFF7EFFF86002800FFF7EBFF830013
:1004F00000209E420ED1231D9E1904351A009E42F3
:1005000007D929781278013301358A42F6D00020C4
:1005100000E0012070BD0000F0B585B003930190AC
:1005200002912D4E2D4B002A02D002223270013A48
:1005300000251A601B68F554019B9D424ADA029A15
:10054000AB00D058254B1C68C8239B0037191C1BD7
:100550000123184202D04310214A1FE0214A0028FB
:1005600002D0042805D1204A2100380004F044FFBD
:1005700018E0042810D90F2302681340042B04D17B
:1005800001F0E6FC194A030008E0062B05D1FFF74D
:1005900099FF174A030001E00123164A21003800A1
:1005A00004F02AFF300004F083FF039B0B4A002B6A
:1005B00001D110600CE0019B013B9D42F9DA0E4B2A
:1005C0009842F6DC431C1360202232540022F2547D
:1005D0000135B1E705B0F0BDFC000020F8000020B7
:1005E000B1630000846300008A630000D0650000EE
:1005F0008F630000A06300001F030000C368F0B514
:100600009D00836887B05D19030018330393036965
:1006100002909C00039B1F1943699E000093039B5B
:100620009E19D64B1B78002B0FD17F222B68D44903
:100630001C1213409B005B5800960435019235E074
:10064000CE4B1B78002B29D0009E029BCB4C9B6885
:1006500021780093EA1A029B92109B7812021A43A7
:10066000029B587802F0DEF90023029A237013707F
:1006700000960497029B039A9B68ED1A0193029BD4
:10068000AD10DD60049B9F1A029BBF101F61009B91
:100690009B1A029A9B10536101F060FB2B68019A30
:1006A0001C121340B64A9B009B5804359F46029B80
:1006B000587802F0AFF90023029A1370D9E7039B30
:1006C0003A1DD11AAD4B8B2903DD1A22009E1A70F8
:1006D000BBE71B783C60002B02D0009E1700B4E7FC
:1006E0002B6801991C120B40A5499B005B58170011
:1006F0000435DBE7039B3A1DD11AA04B8B2903DDA0
:100700001A22009E1A70A0E728681B78291D3860FD
:10071000002B03D0009E17000D0096E76B6801992F
:100720001C120B4096499B005B5817000835BDE72B
:10073000039B3A1DD11A914B8B2903DD1A22009E8F
:100740001A7082E7A4001B782C193C60002B02D0A1
:10075000009E170079E72B6801991C120B4088490D
:100760009B005B5817000435A0E7039B3A1DD11A84
:10077000824B8B2903DD1A22009E1A7065E781489F
:10078000A40021581B783960002B02D0009E17006E
:100790005BE72B6801991C120B4079499B005B5861
:1007A0001700043582E73A1F764B1168A400E15028
:1007B000724B1B78002B02D0009E170045E72B6878
:1007C00001991C120B406E499B005B5817000435C1
:1007D0006CE76C4BA600F058FFF766FE043F040080
:1007E0003868FFF761FE24180120664B640004435B
:1007F000F450624B1B78002B01D0009E25E72B683C
:10080000019A1C1213405E4A9B009B5804354DE729
:10081000039B3A1DD11A594B8B2903DD1A22009EE6
:100820001A7012E70098039C0121A04202D901002E
:100830000C3909681B783960002B02D0009E170024
:1008400003E72B6801991C120B404D499B005B5834
:10085000170004352AE7039B3A1DD11A474B8B2911
:1008600003DD1A22009E1A70EFE600990398814278
:100870000AD90B000C3B1B6843495B106418E41A4F
:10088000009BA400E35802E01821197000233B608C
:100890003A4B1B78002B02D0009E1700D5E62B6840
:1008A00001991C120B4036499B005B581700043518
:1008B000FCE6009B039A93420CD90C3B1968324B1F
:1008C0003A1FE3184910591A1068009B8900C85054
:1008D000170002E01822294B1A70284B1B78002BB6
:1008E00001D0009EB1E62B68019A1C121340244AE5
:1008F0009B009B580435D9E6009B039A934220D96C
:10090000009E214B0C3EE31804933368049A5B105D
:10091000D31A009A9B009858FFF7C6FD3C1F05901C
:100920002068FFF7C1FD3168049B4910591A059BE7
:1009300089001F1801207F00009B0743CF5027002C
:1009400002E018220D4B1A700C4B1B78002B01D0C3
:10095000009E7AE62B68019A1C121340084A9B00FD
:100960009B580435A2E6039B3A1DD11A034B8B29F1
:100970000CDD1A22009E1A7067E6C046F0000020C7
:1009800084610000081A0020FDFFFF3F0099A400C9
:1009900061581B783960002B02D0009E170054E686
:1009A0002B6801991C120B40CD499B005B58170026
:1009B00004357BE63A1F009B1168A400E150C94B47
:1009C0001B78002B02D0009E17003EE62B68019991
:1009D0001C120B40C2499B005B581700043565E6AA
:1009E000009BA4001C192368043F38685E10FFF7C1
:1009F0005BFD36180120BB4B76001B780643266052
:100A0000002B01D0009E20E62B68019A1C12134097
:100A1000B34A9B009B58043548E6039BA4003F1B48
:100A2000B04CBB420DD82378002B01D0009E0CE6C1
:100A30002B68019A1C121340A94A9B009B5804354D
:100A400034E6A94801F0FAF92378002B01D0009E82
:100A5000FBE52B68019A1C121340A14A9B009B588E
:100A6000043523E6A300ED18002C00DA01E69D4BC7
:100A70001B78002B01D0009EE7E52B68019A1C1221
:100A80001340974A9B009B5804350FE63B1F049385
:100A90001B680593042B04D1A300ED18002C00DA89
:100AA000E8E5904B1B78002B02D0009E049FCCE51C
:100AB0002B68019A1C121340894A9B009B58049F83
:100AC0000435F3E53B1F04931B680593002B04D109
:100AD000A300ED18002C00DACCE5824B1B78002B2C
:100AE00002D0009E049FB0E52B68019A1C121340AF
:100AF0007B4A9B009B58049F0435D7E53A1F136837
:100B00005B10013B002B07DD01215B00A4000B43C0
:100B100004972D191360ADE5724B17001B78002B5D
:100B200001D0009E91E52B68019A1C1213406C4A7B
:100B30009B009B580435B9E53A00039B0C32D31A4D
:100B40008B2B04DD1A22674B009E1A707DE5FF2374
:100B500061005B000B4001210B433B60029B03984B
:100B60009B6824120493ED1A029BAD109B782D0212
:100B70001D43009B8D401B1A9B108B400B43BB6099
:100B8000029B0D437D609C70E4B2584BE4000299D7
:100B9000E35816008B6053490978002903D00833C5
:100BA0001D00170051E51D0001999B680C351C12B2
:100BB0000B404B499B005B580092170076E53B1FAA
:100BC0001E68039A009B93422AD104970A20F307D8
:100BD00016D4B3070DD1042E0BD90F23326813405E
:100BE000042B06D1300001F0B3F904F061FC0630AB
:100BF00006E00720042E03D0002E01D080208000C4
:100C0000643001F03FFD002801D1043D32E5029B34
:100C10003100587801F018FF0023029A137029E57B
:100C2000009B009A0C3B1B6802995B109B005B4287
:100C30001C00D3180C3B1E601300083B1B68083CCB
:100C400017195A108A70D2B22849D2005B00555841
:100C50009B0A029A9B009560ED18009B043B1E685E
:100C6000039B7610B6009E191E4B1B78002B00D0FC
:100C7000EBE42B68019A1C121340194A9B009B5805
:100C80000096043512E53B1F1868FFF70DFCA40021
:100C900006003F1B1E2818DC02F04AFC083E3618EE
:100CA00002F046FC124B801B9842F9D80D4B1B7882
:100CB000002B01D0009EC8E42B68019A1C1213403F
:100CC000074A9B009B580435F0E40123029A1370F5
:100CD00002F02EFC029B113886195E60C9E4C04602
:100CE00084610000F0000020B463000010120020B6
:100CF0009F8601003B1F1868FFF7D6FBA4003B1B33
:100D00000493BE4B061E9E4209DC0123029A137017
:100D100002F00EFCFA239B005E43113E04E0022326
:100D2000029A137002F00EFC029B36185E60A1E47A
:100D3000A300FF1A002320001A003900FFF7ECFB84
:100D4000AF4EB04C3168200001F036FE3168200013
:100D500001F081FEAC4B1B78002B01D0009E74E4A7
:100D60002B68019A1C121340A84A9B009B5804351B
:100D70009CE4A54BA4001B783F1B002B01D0009ED8
:100D800063E42B68019A1C121340A04A9B009B58F5
:100D900004358BE401F0BCFC00F0E0FF3B1F186859
:100DA000002823D1083B1868C30701D5401016E07E
:100DB00083070FD104280DD90F2302681340062B97
:100DC00002D1FFF77FFB0AE0052B03D1FFF77AFB87
:100DD000800004E019228C4B009E1A7035E43A0022
:100DE00001214300083A0B43136001E04010013831
:100DF000002832DD012243001343391F0B603B0002
:100E0000083B1B681341181A3B000C3B1B6813423C
:100E100003D08018A400904015E0990717D1042B47
:100E200015D90F211E683140062906D101308000F6
:100E3000C358009AA400A35010E0052907D1181840
:100E40000079A4004000009B1043E05006E0192206
:100E50006D4B009E1A70FFF7F8FB04356A4B1B7848
:100E6000002B02D0009EFFF7F0FB2B68019A1C12AA
:100E70001340664A9B009B58043517E4A300039A6D
:100E8000FB189B1A8B2B01DC002205E01A225E4B1B
:100E9000009E1A70FFF7D9FB631E002C03DD3A6039
:100EA0001C000437F8E7584B1B78002B02D0009E3B
:100EB000FFF7CBFB2B68019A1C121340534A9B008F
:100EC0009B580435FFF7F2FB3B00083B1868FFF71F
:100ED000EBFA3B1F04901868FFF7E6FA049AA600A5
:100EE000BC1B0023824200DA04332360464BBC1B48
:100EF0001B78271D002B02D0009EFFF7A6FB2B6856
:100F0000019A1C121340414A9B009B580435FFF77D
:100F1000CDFBA300FE1A04933B00083B1868FFF7C3
:100F2000C3FA3B1F04001868FFF7BEFAE20FC317AD
:100F3000A04253419B003360049BFC1A324B271D97
:100F40001B78002B02D0009EFFF77FFB2B68019AD5
:100F50001C1213402D4A9B009B580435FFF7A6FB3B
:100F60003B00083B18683B1F1968A300884202D168
:100F7000FB1A042222E004281ED90122104201D0CB
:100F8000114219D10326304215D10F2302681A40AD
:100F9000042A10D131420ED104290CD90A68134019
:100FA000042B08D1FFF79AFA431E9841A600BE1BF6
:100FB0008000306003E0A3000022FB1A1A60124B8D
:100FC000A4001B783C1B271D002B02D0009EFFF7BE
:100FD0003CFB2B68019A1C1213400C4A9B009B5847
:100FE0000435FFF763FB3B00083B18683B1F19689B
:100FF000A30088420CD1FB1A00222DE0E703000079
:10100000F8000020FC000020F000002084610000B7
:1010100004281FD90122104201D011421AD10326FF
:10102000304216D10F2302681A40042A11D13142EE
:101030000FD104290DD90A681340042B09D1FFF7F9
:101040004DFA030058425841A600BE1B8000306094
:1010500003E0A3000422FB1A1A60EA4BA4001B78E9
:101060003C1B271D002B02D0009EFFF7EEFA2B68D9
:10107000019A1C121340E44A9B009B580435FFF769
:1010800015FBA300FE1A04933B00083B1868FFF70A
:101090000BFA3B1F04001868FFF706FAE217C30FAC
:1010A000844253419B003360049BFC1AD54B271D9F
:1010B0001B78002B02D0009EFFF7C7FA2B68019A1D
:1010C0001C121340D04A9B009B580435FFF7EEFAE0
:1010D0003B00083B1868FFF7E7F93B1F04901868CE
:1010E000FFF7E2F9049AA600BC1B0023824200DD50
:1010F00004332360C34BBC1B1B78271D002B02D07D
:10110000009EFFF7A2FA2B68019A1C121340BE4AF8
:101110009B009B580435FFF7C9FA3B1F1B68B94A6F
:10112000A400042B02D13B1B002103E0002B03D1C0
:1011300004213B1B196001E00C23137013783C1B46
:10114000271D002B02D0009EFFF77FFA2B68019A23
:101150001C121340AC4A9B009B580435FFF7A6FABB
:10116000A300FC1A04933B00083B1868FFF79CF9A6
:101170003B1F06001868FFF797F936180120049BFB
:10118000760006432660FC1A9E4B271D1B78002B19
:1011900002D0009EFFF759FA2B68019A1C121340E7
:1011A000994A9B009B580435FFF780FAA300FE1A6A
:1011B00004933B00083B1868FFF776F93B1F0400D7
:1011C0001868FFF771F9241A0120049B6400044396
:1011D0003460FC1A8B4B271D1B78002B02D0009E1D
:1011E000FFF733FA2B68019A1C121340864A9B00C2
:1011F0009B580435FFF75AFAA300FC1A04933B00EE
:10120000083B1868FFF750F93B1F06001868FFF706
:101210004BF946430120049B760006432660FC1AE6
:10122000784B271D1B78002B02D0009EFFF70DFA8C
:101230002B68019A1C121340734A9B009B5804357B
:10124000FFF734FA3B00083B1868FFF72DF93B1F06
:1012500004901868FFF728F90100049803F064FB74
:10126000012340001843674BA4001B783E1B3060ED
:10127000371D002B02D0009EFFF7E7F92B68019A7B
:101280001C121340604A9B009B580435FFF70EFA6E
:101290003B00083B1868FFF707F93B1F04901868EC
:1012A000FFF702F90100049803F024FC0123490030
:1012B0001943544BA4001B783E1B3160371D002B93
:1012C00002D0009EFFF7C1F92B68019A1C1213404F
:1012D0004D4A9B009B580435FFF7E8F93B1F1868FF
:1012E000FFF7E2F8C317C018584001234000184325
:1012F000444BA4001B783E1B3060371D002B02D0EE
:10130000009EFFF7A2F92B68019A1C1213403E4A77
:101310009B009B580435FFF7C9F9A300FE1A0593FB
:101320003068012C03D1FFF7BFF8049008E0FFF705
:10133000BBF804007068FFF7B7F80130031B049393
:10134000049B002B01DC0123049304F007F80499AB
:1013500003F0D0FB0C190121059B64000C433460A1
:10136000FC1A284B271D1B78002B02D0009EFFF78C
:101370006CF92B68019A1C121340234A9B009B585E
:101380000435FFF793F9A4003E1B3000FFF734F853
:101390001C4B30601B78371D002B02D0009EFFF7DE
:1013A00054F92B68019A1C121340174A9B009B5852
:1013B0000435FFF77BF9A300FE1A04933B00083BBA
:1013C0001868FFF771F83B1F04001868FFF76CF806
:1013D00004400120049B640004433460FC1A094B60
:1013E000271D1B78002B02D0009EFFF72EF92B68DB
:1013F000019A1C121340044A9B009B580435FFF7C6
:1014000055F9C046F000002084610000A300FC1ADA
:1014100004933B00083B1868FFF746F83B1F0600A3
:101420001868FFF741F806430120049B7600064345
:101430002660FC1ADE4B271D1B78002B02D0009E75
:10144000FFF703F92B68019A1C121340D94A9B003D
:101450009B580435FFF72AF9A300FC1A04933B00BC
:10146000083B1868FFF720F83B1F06001868FFF7D5
:101470001BF846400120049B760006432660FC1AB8
:10148000CB4B271D1B78002B02D0009EFFF7DDF809
:101490002B68019A1C121340C64A9B009B580435C6
:1014A000FFF704F93B1F1868FEF7FEFFC043012356
:1014B00040001843BE4BA4001B783E1B3060371D14
:1014C000002B02D0009EFFF7C0F82B68019A1C1277
:1014D0001340B84A9B009B580435FFF7E7F8A30078
:1014E000FE1A04933B00083B1868FEF7DDFF3B1F24
:1014F00004001868FEF7D8FF8440012364001C43F1
:10150000049B3460FC1AAA4B271D1B78002B02D0C9
:10151000009EFFF79AF82B68019A1C121340A54A07
:101520009B009B580435FFF7C1F8A300FE1A0493F3
:101530003B00083B1868FEF7B7FF3B1F0400186824
:10154000FEF7B2FF0441012364001C43049B346096
:10155000FC1A974B271D1B78002B02D0009EFFF72B
:1015600074F82B68019A1C121340924A9B009B58F6
:101570000435FFF79BF8A4003E1B3000FEF757FE32
:101580008B4B30601B78371D002B02D0009EFFF77D
:101590005CF82B68019A1C121340864A9B009B58EA
:1015A0000435FFF783F8A4003E1B3000FEF74FFE22
:1015B0007F4B30601B78371D002B02D0009EFFF759
:1015C00044F82B68019A1C1213407A4A9B009B58DE
:1015D0000435FFF76BF8A4003F1B3800FEF749FE07
:1015E000734B1B78002B02D0009EFFF72EF82B6860
:1015F000019A1C1213406F4A9B009B580435FFF759
:1016000055F8A4003E1B3000FEF765FE684B3060C5
:101610001B78371D002B02D0009EFFF716F82B68B1
:10162000019A1C121340634A9B009B580435FFF734
:101630003DF8A4003F1B3800FEF784FE5C4B1B788E
:10164000002B02D0009EFFF700F82B68019A1C12B5
:101650001340584A9B009B580435FFF727F8A40015
:101660003E1B3000FEF7A8FE514B30601B78371D43
:10167000002B02D0009EFEF7E8FF2B68019A1C1297
:1016800013404C4A9B009B580435FFF70FF8039A10
:101690003B1D0493464C9B1A8B2B04DD1A23009EA2
:1016A0002370FEF7D2FF01F04DFF012340001843E5
:1016B00023783860002B03D0009E049FFEF7C5FFFF
:1016C0002B68019A1C1213403A4A9B009B58049FB6
:1016D0000435FEF7EBFF039A3B1D0493344C9B1A31
:1016E0008B2B04DD1A23009E2370FEF7AEFF01F062
:1016F0001FFF314B40001840012318432378386006
:10170000002B03D0009E049FFEF79FFF2B68019AD9
:101710001C121340274A9B009B58049F0435FEF778
:10172000C5FFA4003E1B3000FEF78AFE204B306050
:101730001B78371D002B02D0009EFEF786FF2B681A
:10174000019A1C1213401B4A9B009B580435FEF75C
:10175000ADFFA4003F1B3800FEF78AFE144B1B7838
:10176000002B02D0009EFEF770FF2B68019A1C121E
:101770001340104A9B009B580435FEF797FFA300C7
:10178000FB1A0493012320001A000499FEF7C4FEFB
:101790000A4C2068643000F075FF002800D1AFE2E9
:1017A000029B21685A78064801F063F91EE0C046A2
:1017B000F000002084610000FEFFFF7FF8000020A1
:1017C000FC000020A300FB1A049320000123002248
:1017D0000499FEF7A1FEE34C2068643000F052FF4C
:1017E000002800D18CE2E04801F066F80223029A5A
:1017F000137001F0A7FE236805331818029B586088
:10180000FEF738FFA4003E1B300001F0BBFED74BB3
:1018100030601B78371D002B02D0009EFEF715FFAD
:101820002B68019A1C121340D14A9B009B58043527
:10183000FEF73CFFA4003E1B300001F0A5FECB4BA1
:1018400030601B78371D002B02D0009EFEF7FDFE96
:101850002B68019A1C121340C54A9B009B58043503
:10186000FEF724FFA4003E1B300001F08FFEBF4BAB
:1018700030601B78371D002B02D0009EFEF7E5FE7E
:101880002B68019A1C121340B94A9B009B580435DF
:10189000FEF70CFFA4003F1B380001F095FEB34B90
:1018A0001B78002B02D0009EFEF7CFFE2B68019A1A
:1018B0001C121340AE4A9B009B580435FEF7F6FEFF
:1018C000A4003E1B300001F0A1FEA84B30601B7845
:1018D000371D002B02D0009EFEF7B7FE2B68019A41
:1018E0001C121340A24A9B009B580435FEF7DEFEF3
:1018F000A4003F1B380001F0BBFE9C4B1B78002B63
:1019000002D0009EFEF7A1FE2B68019A1C12134024
:10191000974A9B009B580435FEF7C8FE0121200022
:1019200001F08EFE914B1B78002B02D0009EFEF73B
:101930008CFE2B68019A1C1213408D4A9B009B5809
:101940000435FEF7B3FE0021200001F079FE874B3D
:101950001B78002B02D0009EFEF777FE2B68019AC1
:101960001C121340824A9B009B580435FEF79EFED2
:10197000A4003E1B300001F0AFFE7C4B30601B78B2
:10198000371D002B02D0009EFEF75FFE2B68019AE8
:101990001C121340764A9B009B580435FEF786FEC6
:1019A000A4003E1B300001F0ABFE704B30601B7892
:1019B000371D002B02D0009EFEF747FE2B68019AD0
:1019C0001C1213406A4A9B009B580435FEF76EFEBA
:1019D000A4003F1B380001F057FE644B1B78002B1E
:1019E00002D0009EFEF731FE2B68019A1C121340B4
:1019F0005F4A9B009B580435FEF758FEA4003F1B2E
:101A0000380001F025FF594B1B78002B02D0009EB7
:101A1000FEF71BFE2B68019A1C121340544A9B00D0
:101A20009B580435FEF742FEA4003E1B300001F037
:101A30004FFF4E4B30601B78371D002B02D0009EAD
:101A4000FEF703FE2B68019A1C121340484A9B00C4
:101A50009B580435FEF72AFEA4003F1B380001F016
:101A6000B9FE424B1B78002B02D0009EFEF7EDFD25
:101A70002B68019A1C1213403D4A9B009B58043569
:101A8000FEF714FEA4003E1B300001F0B9FE374BF8
:101A900030601B78371D002B02D0009EFEF7D5FD6D
:101AA0002B68019A1C121340314A9B009B58043545
:101AB000FEF7FCFDA4003F1B380001F0A1FB2B4BFF
:101AC0001B78002B02D0009EFEF7BFFD2B68019A09
:101AD0001C121340264A9B009B580435FEF7E6FD76
:101AE000A4003F1B380001F097FB204B1B78002B14
:101AF00002D0009EFEF7A9FD2B68019A1C1213402C
:101B00001B4A9B009B580435FEF7D0FDA4003F1BE9
:101B1000380001F08DFB154B1B78002B02D0009E86
:101B2000FEF793FD2B68019A1C121340104A9B008C
:101B30009B580435FEF7BAFDA4003F1B380001F0A6
:101B400093FB0A4B1B78002B02D0009EFEF77DFD15
:101B50002B68019A1C121340054A9B009B580435C0
:101B6000FEF7A4FDF8000020FC000020F00000209B
:101B700084610000A4003E1B300001F047FF784B59
:101B800030601B78371D002B02D0009EFEF75DFDF4
:101B90002B68019A1C121340724A9B009B58043513
:101BA000FEF784FDA4003E1B300001F037FF6C4BB4
:101BB00030601B78371D002B02D0009EFEF745FDDC
:101BC0002B68019A1C121340664A9B009B580435EF
:101BD000FEF76CFDA4003E1B300001F027FF604BB8
:101BE00030601B78371D002B02D0009EFEF72DFDC4
:101BF0002B68019A1C1213405A4A9B009B580435CB
:101C0000FEF754FDA4003E1B300001F007FE544BCC
:101C100030601B78371D002B02D0009EFEF715FDAB
:101C20002B68019A1C1213404E4A9B009B580435A6
:101C3000FEF73CFDA4003F1B380001F031FB484B90
:101C40001B78002B02D0009EFEF7FFFC2B68019A48
:101C50001C121340434A9B009B580435FEF726FD97
:101C6000A300FF1A3900200001F0FCFB3C4B1B785D
:101C7000002B02D0009EFEF7E8FC2B68019A1C1294
:101C80001340384A9B009B580435FEF70FFDA40013
:101C90003E1B300001F0B2FB314B30601B78371D2A
:101CA000002B02D0009EFEF7D0FC2B68019A1C127C
:101CB00013402C4A9B009B580435FEF7F7FCA30009
:101CC000FF1A3900200001F05FFB254B1B78002B29
:101CD00002D0009EFEF7B9FC2B68019A1C1213403B
:101CE000204A9B009B580435FEF7E0FCA4003B1BF8
:101CF0001800049301F048FD01F04BFD022802DCBE
:101D0000043DFEF7B6FC164B1B78002B03D0009E5B
:101D1000049FFEF79AFC2B68019A1C121340114A8B
:101D20009B009B58049F0435FEF7C0FCA4003E1B9B
:101D3000300001F030FD0A4B30601B78371D002B5E
:101D400002D0009EFEF781FC2B68019A1C12134002
:101D5000044A9B009B580435FEF7A8FC07B0F0BD71
:101D6000F000002084610000014B187000207047D3
:101D7000F0000020F0B50023A02787B05A1E04927F
:101D8000002B05DC01F0F0F800F07CFE1923049331
:101D9000002503950295254B19688D4201DB049BB4
:101DA000ECE7234B1A680132914200DC00221A60F2
:101DB0001B68204E01937B439A199B5D059234006A
:101DC000032B01D110002CE0002B2DD0012B0CD1C6
:101DD000029B002B02D101F0ABFB0290019A029909
:101DE0007A43A4186368CB1A0FE0022B12D1039B2D
:101DF000002B02D101F0A6FB0390019A03997A43CC
:101E0000A4186368CB1A9B029B0A0B498B4201D82A
:101E10000323B354019B074A7B439B5C032B03D1F1
:101E20000598FEF7EBFBBAE70135B4E7F4000020B4
:101E300000000020D00B00209F86010000B59BB061
:101E40000200054901A803F009FB01A800F034FDD8
:101E500000F018FEFCE7C046C463000037B5174D1C
:101E600004002868002801D002F0ECFEA400200045
:101E700002F0DEFE2860002801D1114809E001AB24
:101E8000984208D20F4B02196B440193934202D23D
:101E90000D48FFF7D3FF042802D808302860083C1B
:101EA0002B680A4A1C191360094B01211C6000238E
:101EB000084AD1500433642BFBD137BD24040020E1
:101EC000D56300001CFCFFFF056400001C0400201B
:101ED00020040020081A002070B50D4D0D4E2B680F
:101EE0004C1CA40036681C19B44203D90A20FFF721
:101EF0003BFF0BE02C601D00AC4201D904C5FBE7A1
:101F00000F220901104008431860180070BDC04638
:101F10001C040020200400200322CB1C70B50C0000
:101F2000D9171140C9180500891000220420FFF7B5
:101F3000D3FF0023A34204DAE95CC2181171013314
:101F4000F8E7E1430023C917214041180B7170BD28
:101F500010B5830706D1042804D90F2304C8134001
:101F6000042B03D00E20FFF7FFFE014810BDC04632
:101F70000C65000030B502248025094B094AED00AC
:101F80009C505C59002CFCD0A124E400884204D26F
:101F90008025ED0018514019F8E70021995030BD17
:101FA00000E001400405000010B5002804D1902095
:101FB00092210002890203E0922080218002C9025E
:101FC000FFF7D8FF10BD002802D092239B0201E04A
:101FD00090231B021B6800201A0E532A01D11B02FA
:101FE000180A704730B501248025064A064BED00DB
:101FF000D4505459002CFCD001600021014AD1502A
:1020000030BDC04600E001400405000010B50028C6
:1020100002D09220800201E090200002A623090253
:10202000DB05090A1943FFF7DDFF10BDF0B50124F8
:10203000802503000F4F08000F49ED007C507C59AC
:10204000002CFCD09C46002810DD5478167893783C
:10205000240234431B0423431C00D37801381B069D
:102060002343644608C40432A446ECE700237B50B3
:10207000F0BDC04600E001400405000070B5050059
:102080004B680A009C1C2100FFF7D0FFA000281815
:1020900070BD0000154B1B68002B04D080219223DB
:1020A000C9029B0203E09221902389021B020028AF
:1020B00007D1191D5B6802001B0E522B14D10A00B8
:1020C00012E0002281420FD903681B0E522B0BD164
:1020D000436802339B00C318994205D91A68110E50
:1020E0000022522900D11A00100070472806002053
:1020F0008022F0B5520085B00021624802F0B5FDA3
:10210000802200215200604802F0AFFD5F4B1B6847
:102110001A00029353425A4110000392FFF744FF02
:10212000029B002B01D15A4C00E05A4C0020FFF7D3
:10213000B1FFFF270500002D00D194E02B681A1293
:102140001B143A403B4001921A000A3A092A43D82C
:102150004C4B019A995C002900D07FE010224E4838
:1021600002F083FD2E00336801991A123A40914221
:1021700017D11A143A400B2A06D0132A0CD00A2A77
:102180000FD1454B1E600CE03B40022B09DC424A5C
:102190009B00D3185E6004E0102200213E4802F04C
:1021A00064FD3000FFF776FF061EDCD13A4B19685C
:1021B00000290FD02000FFF761FF0400374E31687F
:1021C000002903D02000FFF759FF0400344B0436E8
:1021D000B342F4D12B4B3EE0143B092B3ED82A4BA3
:1021E000019A995C002939D108222E4802F03DFD60
:1021F0002E0033681A143A40152A0BD01D2A11D02C
:10220000142A14D1019A1B123B409A420FD1254B3C
:102210001E600CE0019A1B123B409A4207D1214BF1
:102220005E6004E0082200211E4802F01EFD30001E
:10223000FFF730FF061EDCD11A4E3168002909D0A5
:102240002000FFF71BFF71680400002902D0FFF790
:1022500015FF04000C4B0121019A99542800FFF747
:1022600019FF050067E70298FFF7ADFE411C0398D0
:10227000FFF7CCFE054B039A1A600B4B1C6005B0B0
:10228000F0BDC046280500202804002028060020B4
:1022900004480200049000006C1A0020701A00200C
:1022A0007C1A00207C1A00202C06002070B500202B
:1022B000FFF789FE04000120FFF785FE844200DA63
:1022C00004000A4B1E687542754128001D60FFF727
:1022D0006BFE002E01D0064B00E0064B064A28009C
:1022E000611C1360FFF792FE70BDC04628060020F7
:1022F00004900000044802002C060020F8B50020DD
:10230000FFF761FE07000120FFF75DFE3E00224D52
:102310000643224C0CD180219020C9020002FFF715
:1023200029FE01213000FFF771FE2E601C4B2FE0CB
:10233000874208DD002392212B60194B890223601C
:102340002368002011E0012380212B60154BC90276
:102350002360F5E71A68551C18D0120E522A07D1CF
:1023600001205A68023292009B188B42F2D311E08E
:10237000002800D023600C4C0C49200003F090F89A
:10238000200001F0E5F8FFF791FF04E0002802D0FB
:10239000236000E02160F8BD280600202C06002004
:1023A0000490000004480200841E00207D640000A8
:1023B000F0B585B0039203220333DC171440294E95
:1023C000E3189C10336801900291002B02D0802208
:1023D000D20201E092229202234FA51C3B68AD007D
:1023E0005B199A4217D2FFF783FE3368002B02D0A5
:1023F0008022D20201E0922292023B685B199A424B
:1024000009D21A4C1A49200003F04AF8200001F0C2
:102410009FF8002023E0029B3E681B06190C6B46C8
:102420001A7BA423DB051343019A0B431104FF22FB
:102430001204114019433000FFF7D4FD3300301D62
:10244000083321000193FFF7CDFD01980A9A21007E
:10245000FFF7ECFD3000019B083D5D193D6005B0C4
:10246000F0BDC046280600202C060020841E002057
:10247000A664000070B59AB0FFF740FFFF221F4C22
:10248000D2000021200002F0F0FB0020FFF702FE46
:10249000FF25002600281AD003681A142A400A2AA9
:1024A00008D11A122A40FF2A0ED0D200A1180B71AF
:1024B000A05009E0132A07D11B122B40FF2B03D099
:1024C000DB00E2181671E650FFF7E4FDE2E7FF21BA
:1024D0000200C900235808305D1EAB41D218884263
:1024E000F8D1074901A802F0B9FF01A800F0E4F90A
:1024F000044800F0E1F91AB070BDC0461012002087
:10250000CD640000E5640000044A05491368C8541E
:1025100001339B059B0D13607047C046300A0020B5
:1025200030060020114A70B51368114C984211DA38
:1025300006193178451CFA39012905D8AB4205DD69
:10254000717801391F2901D92800EFE70100251A08
:10255000461C02D10023136006E0665C6E54013114
:102560008B42FADC181A106070BDC046340A002095
:10257000841A002010B500F0DBFF064B1A68904269
:1025800001D200221A601B68C01A034B83428041AB
:10259000404210BD380A0020204E000010B5094A04
:1025A000094C1268236893420AD0084AD05C01F0B3
:1025B000E3F8012804D1236801339B059B0D2360B8
:1025C00010BDC046300A00203C0A00203006002022
:1025D00010B50400064B074A1B6812689B1ADB43C0
:1025E0009B059B0DA34202DAFFF7D8FFF2E710BD6F
:1025F000300A00203C0A0020F7B506000191151EA4
:102600002FD05768B800441C0630FFF7E1FFFB20CD
:10261000FFF77AFF1C20FFF777FFF0B2FFF774FF98
:10262000E0B22412FFF770FFE0B2FFF76DFF6B46D8
:102630001879FFF769FF0026BE4212DAB300EB18E3
:102640009C680136E0B2FFF75FFF2012C0B2FFF7CF
:102650005BFF2014C0B2FFF757FF200EFFF754FFB7
:10266000EAE7F7BDC82210B5D2000021034802F006
:10267000FCFA0022024B1A6010BDC046D00B0020AD
:10268000F4000020064B074A1B6812689B1ADB43C4
:102690009B059B0D0122834200DC00221000704745
:1026A000300A00203C0A0020F8B505000C00160096
:1026B0001F1E0ED10320FFF7E5FF002827D0FA20C8
:1026C000FFF722FFE8B2FFF71FFFE0B2FFF71CFFA2
:1026D0001DE0501DFFF7D6FF002818D0FB20FFF7A4
:1026E00013FFE8B2FFF710FFE0B2FFF70DFFF0B203
:1026F000FFF70AFF3012C0B2FFF706FF3C00E31BF2
:102700009E4204DD2078FFF7FFFE0134F7E7F8BDB5
:1027100070B50024A0250B4B1B689C420EDA2A00E2
:102720006243094BD3181A78002A05D05978002340
:1027300011201A00FFF7B8FF0134ECE7FFF792FF12
:1027400070BDC046F4000020D00B00200123F3B57B
:102750000400FFB00D0010001A420DD002AA137041
:10276000431002A9537042121B0E40148A700B7161
:10277000C8700B00052273E0032313401ED1042A06
:102780001CD90F2201680A40042A17D1023302AA79
:102790001370FFF7DDFB060002F08AFEF823FF331B
:1027A000984200DD18000023834205DA01335A1EE7
:1027B000B25C02A9CA54F7E7421C50E0042801D0D9
:1027C000002809D1032302AA04381370434243416D
:1027D00053701300022243E0002B45D1042843D953
:1027E0000F2102681140052912D1043302A90B7090
:1027F000F8231209FF3392009A4200DD1A000023E9
:1028000093422BDA0133C118C97802AEF154F7E7CD
:10281000062929D101390E00120956430196F826DE
:10282000019FFF36B7421FDC02AE31700136934282
:1028300013DA0127013399004158394201D0394157
:1028400000E00A49012737700F127170B7700F143A
:10285000090EF77031710536E9E7019A013202ABD2
:1028600029002000FFF720FF7FB0F3BD19FCFFFF18
:1028700070B5A023050000240D4A1800604380189D
:102880004178A94203D001340A2CF6D10FE0A022EE
:10289000002102F0EAF9074A1368013BA34200D184
:1028A0001460002329001A001120FFF7FDFE70BDFF
:1028B000D00B0020F400002010B5B2B002236A460D
:1028C0000400137002F0F4FDC72800DDC7200023C8
:1028D000834205DA694601335A1EA25CCA54F7E7FF
:1028E000421C6B46FF211420FFF7DEFE32B010BD04
:1028F000F7B5234B06001B68A02000930023214955
:10290000009A93420ADA02005A438A185478B44271
:1029100002D11278002A32D10133F1E70024A0233A
:102920001A00624301920199164A55182F78002F18
:1029300006D001340A2CF3D11348FFF7BDFF1EE087
:10294000A0223900280002F090F903230D4A0199D2
:102950006E7053540D4BF200D358AE70AB6002232F
:10296000EB60009B2F616F61A34202DC044B0134DA
:102970001C60002331001A001020FFF795FEF7BD00
:10298000F4000020D00B0020A065000010120020F1
:1029900010B5FFF7BDFE0024064BE200D3181B79EB
:1029A000043B012B02D8E0B2FFF7A2FF0134FF2C59
:1029B000F2D110BD10120020F8B507000D00002460
:1029C000134BE200D3181A79062A1DD11868793200
:1029D000C3681A40042A17D11B0A01339B000C302C
:1029E000C018FFF7B5FA060002F062FD0023A84206
:1029F0000AD19D4205DDF15CFA5C914204D10133BC
:102A0000F7E7E0B2FFF774FF0134FF2CD8D1F8BD2F
:102A100010120020002310B501001A001120FFF74A
:102A200043FE10BD07B56B46197069465A70131204
:102A30008B701314120ECB700A716B4601000522C5
:102A40001320FFF731FE07BD10B50A000100122068
:102A5000FFF77CFE10BD70B5050008000C00323099
:102A6000FFF7B6FD2B00220000211B20FFF71CFE04
:102A700070BD10B50C000300110014202200FFF7F8
:102A800013FE10BDF0B580279DB0FFF787FDB14C58
:102A9000B14D2068FF00391A401900F053FE236839
:102AA0000600C3182360002B00D10BE2002E0DDDC1
:102AB0002068391A281800F045FE236806001B1804
:102AC000236000F035FDA54B1860EFE72B78FA2B5B
:102AD00000D051E12368022B06DCFFF74BFD0028F4
:102AE00000D1EFE10120E6E16878AC7802381828DF
:102AF00000D92CE101F084FE19002A002E003200DA
:102B0000350039002B014400850094009A00AE0086
:102B1000FF0014012B012B012B012B012B012B0199
:102B20002B012B012B012B012501FF2C00D10EE1E4
:102B30002000FFF79DFE00228949E3005A50CB1880
:102B40001A71210000921300132066E02000FFF7A5
:102B5000CFFEFCE02000FFF78BFEF8E0FFF718FF48
:102B6000F5E0FFF7D5FD7F48E8E0182C00D9EEE04E
:102B70007D4BA200D25821001520FFF7E7FDE6E0CB
:102B800000260020FFF786FA00250400002C12D052
:102B9000FF2123681A140A40152A04D11B120B4086
:102BA000B34203D18AE11D2A00D100252000FFF79E
:102BB00071FA0400EAE7002D03D10136192EE0D1A5
:102BC000C5E02800083002F073FC07000530FFF76D
:102BD000FFFCFB20FFF798FC1D20FFF795FCF0B2EF
:102BE000FFF792FCF8B2FFF78FFC3812C0B2FFF784
:102BF0008BFCA742E1DD2B19187AFFF785FC013425
:102C0000F7E700230121584AD1500433642BFBD14C
:102C100000211D200B000A000091FFF7C9FB96E080
:102C200000222100009213002720F6E700F098FC14
:102C300003AC4E4A642100904D4B200002F0DCFBB7
:102C400002232000237002F033FC23000200002145
:102C500016207AE00024424AE300D558002D46D0E1
:102C60006B689E00701DFFF7B3FC2B00002532003F
:102C7000083321000120FFF717FD0020FFF70AFAB3
:102C80002E002F0000281DD0FF2103681A120A40D1
:102C9000A24214D11A140A400B2A07D10B400DD0BE
:102CA000012B09D0022B00D10AE108E0132A06D13A
:102CB00000252E002F0002E0060000E00700FFF7CD
:102CC000E9F9DFE7002E04D0320001212000FFF7F0
:102CD00093FC002D04D02A0002212000FFF78CFC79
:102CE000002F04D03A0000212000FFF785FC0134BA
:102CF000FF2CB0D12BE0FFF70BFD002500242900AD
:102D000000942300220013200135FFF751FBFF2D13
:102D1000F4D1FF222100D200114801F0A6FF16E0F5
:102D2000FFF7F6FC002000F077FA00F01DF900F044
:102D3000FBFCE120C000FFF791F80E48FFF7BCFD57
:102D400005E000231A201A001900FFF7ADFC03204C
:102D5000B1E0C046340A0020841A0020380A00205E
:102D600010120020B5650000081A0020CC65000094
:102D7000C7650000D3650000FB2B00D0B2E62268D7
:102D8000042A00DCA9E62E79E8784F4B3602064388
:102D90009E4200DDA6E6331D9A4200DC9DE6EB5C18
:102DA000FE2B00D09EE66878AC78731E1C2851D0AC
:102DB00006D808281ED01B2847D001287AD105E064
:102DC0001E2869D051D31F286CD073E0FF2C71D01E
:102DD0002000FFF74DFD6D793C4AB31E00922100A3
:102DE0002A000A20FFF7E4FA394BE400E0501C19EE
:102DF00025715FE0182C5DD86879022813D003286C
:102E00001BD0012856D1AF1D7A78AD79BB7812025C
:102E10002A431B0413431A00FB78A4001B06134328
:102E20005B0003430EE0002B44DDB11E2748FFF793
:102E300073F8284BA400E0503CE0AB79A4005A1E84
:102E400093419B00234AA35034E019002248FFF726
:102E5000B3FD2FE0FF2C2DD06A79022A2AD81B4916
:102E6000B31E00910B20210022E0632B00DD6323C1
:102E7000002203A8934204DDA91849798154013244
:102E8000F7E7D9430022C917194041180A700133E6
:102E90000090210015200BE00F4A210000921E2017
:102EA000002205E0042B05D10B4A210000920022EC
:102EB000FFF77EFA701DFFF735FB03E0250075E68E
:102EC0000500FCE61DB0F0BDF60300008A1A0020E4
:102ED00010120020081A0020891A0020F0B5EFF324
:102EE00010810123194083F31088134E134AB4460E
:102EF0001268013A9340124A1468124A1568124A3D
:102F0000002B15D0166803420BD02660C046C04681
:102F1000C046C046C046C046C046C04616682E6081
:102F200004E067463E601668084F3E605B08E7E7CE
:102F300081F31088F0BDC046080500500400002051
:102F4000480A0020500A0020400A00200C050050CA
:102F500010B50124044001D0441002E00D20FEF71A
:102F600003FF200010BD0000F0B5A14F85B03B6805
:102F7000002B04D19F4A1268002A00D136E19E4DF1
:102F80002A68002A2AD19B4E3468002C0FD1002BCE
:102F90000DD00C32994901A801F05EFE6B46043356
:102FA000185D0121013400F0DFFA0C2CF6D13368F2
:102FB000002B11D03C68002C0ED101AD0C228F49A2
:102FC0002800346001F048FE285D0021013400F043
:102FD000CBFA0C2CF8D109E13B68336000211A20B0
:102FE00001F0FEF800211B2001F0FAF800211C205E
:102FF00001F0F6F82E68012E56D0022E00D19CE08A
:10300000002E00D0ECE0013631007A4C032023681A
:10301000994301F0E5F80420216801400B00594272
:10302000594101F0DDF8102123680A200B40594274
:10303000594101F0D5F88021236809010B4059421C
:103040005941062001F0CCF88021236809020B4089
:1030500059425941072001F0C3F8802123684902F1
:103060000B4059425941092001F0BAF880212368E8
:1030700089020B4059425941192001F0B1F88021D1
:103080002368C9020B4059425941182001F0A8F8A1
:10309000802321681B030B4059425941172001F03E
:1030A0009FF831001A2099E00221524C1720236822
:1030B0000B405942594101F093F808212368182028
:1030C0000B405942594101F08BF880212368C90017
:1030D0000B4059425941042001F082F880212368B5
:1030E00049010B40594259410A2001F079F88021E9
:1030F0002368C9010B4059425941032001F070F87F
:103100008021236889030B4059425941092001F06D
:1031100067F8802321681B040B405942594119204C
:1031200001F05EF83100062001F05AF83100072066
:1031300001F056F831001B2050E020212D4C1720C3
:1031400023680B405942594101F04AF84021236855
:1031500018200B405942594101F042F88021236860
:1031600019200B405942594101F03AF88021236857
:1031700049000B4059425941092001F031F88021A2
:10318000236889000B4059425941072001F028F873
:103190008021236889010B4059425941062001F0E2
:1031A0001FF88021236849030B40594259410A20E6
:1031B00001F016F880212368C9030B405942594198
:1031C000032001F00DF8802321685B040B40594275
:1031D0005941042001F004F801211C2001F000F8FD
:1031E0002B680321581C01F085FC296005B0F0BD57
:1031F0004C0A0020440A0020540A0020EB6500001D
:10320000006810B5C30703D5FFF7A2FE014B186095
:1032100010BDC0464C0A002013B5002401A801943B
:1032200000F032FA014B1C6013BDC0464C0A00206E
:1032300070B505000068FFF78BFE04006868FFF7B3
:1032400087FE631E042B0CD80138042809D80522F8
:103250005043043AC3189A40130002490A681343C2
:103260000B6070BD4C0A002070B505000068FFF7C8
:103270006FFE04006868FFF76BFE631E042B0CD81A
:103280000138042809D805225043043AC3189A404B
:10329000130002490A689A430A6070BD4C0A002074
:1032A000F7B5304A1368002B0CD12F4B1968012356
:1032B0008B402E490B602E4911602E4A2E49116019
:1032C0002E4A136001260468344219D0FF2263108D
:1032D000180212041040FF22611212020A40DBB2EF
:1032E00010431843264B1B68202B06D1B440254BB6
:1032F000A40EA400E35800021843FFF7EFFD30E0EE
:10330000032525402DD1042C2BD90F2322681340EF
:10331000062B26D1FF27130901933F04019B9D42F1
:103320001FDAAB00E3185A68324218D05310180263
:103330003840FF2184460902501208406146DBB242
:10334000084318430E4B1B68202B06D15200920EE7
:103350000C4B9200D35800021843FFF7BFFD013514
:10336000DCE7F7BD480A0020CC690000400A0020D5
:1033700008050050500A00200C05005018050050A8
:1033800004000020F8650000012310B50C68134A02
:10339000234003D06310012804DC07E001281ADD74
:1033A00001235B4248682021042800D018211160C5
:1033B000202B00D900230A4A9B009A5801239340EE
:1033C000084A09491360094A1160094A094911600C
:1033D000094A136010BD18211160ECE704000020B9
:1033E000CC690000400A002008050050480A00206F
:1033F000500A00200C050050180500500068F8B570
:10340000C30702D5FFF7A4FD0BE0830726D10428EC
:1034100024D90F2203681A40042A1FD11B091DD08A
:1034200000790300203B5E2B18D80522002053436F
:103430000B4E9D18043AAB420CD0052110249F5D21
:103440003C4200D080180139520064100029F7D1A5
:103450000133F0E701234000184300E00120F8BDEC
:10346000F8660000F0B5040085B008680E00FFF7AC
:103470006FFD0190022C07DD7068FFF769FD040005
:10348000B068FFF765FD01E001200400174B011D46
:103490001A680523461E43430120002784460291F3
:1034A000211D053B039102998E4219D0611E039D97
:1034B000A94212D0042E0DD804290BD8019D5F1803
:1034C000054203D06546BD402A4302E06546BD4043
:1034D000AA43012740000131E9E701360533E2E75D
:1034E000002F01D0014B1A6005B0F0BD4C0A00203E
:1034F00010B50A2000F0FAFC0023FF21024A99547B
:1035000001331D2BFBD110BD580A002001220020E1
:10351000054B06491A615850033004315850801841
:10352000083158501A6070470080004004050000C0
:103530000122034B1A64A822D20098587047C04653
:103540000080004010B5FFF7F3FF800A10BD0000B7
:1035500010B50100014800F0FDFE10BD5C0B00201D
:1035600000487047D368000070B5054E0400335C16
:103570000D008B4202D000F015FE355570BDC046DF
:10358000580A00200D2070473B207047036870B533
:103590005B100120052B12D8094A9B009C58094D4D
:1035A0002B5D002B05D00021200000F0FBFD002347
:1035B0002B55200000F0A0FC01234000184370BDF3
:1035C000E0680000580A002070B5036845685C1088
:1035D0006D1004D40B4B9D4202DD1D0000E0002560
:1035E0001C2C0DD8084E335D012B05D00121200085
:1035F00000F0D8FD012333552900200000F00AFD1A
:1036000070BDC046FF030000580A002070B5046872
:1036100064101C2C0FD8094D2B5D002B05D0002108
:10362000200000F0BFFD00232B55200000F0EEFD30
:103630000423012800D00023180070BD580A002080
:1036400070B504000D001C280ED8084E335C012B09
:1036500004D0012100F0A6FD0123335529002000EC
:103660004D1EA94100F0BCFD70BDC046580A0020A7
:10367000436810B5191F4A424A41006811004010C2
:10368000FFF7DEFF10BD000070B5124C0500A37EF1
:10369000012B05D001211A2000F084FD0123A3761F
:1036A0002379012B05D00121042000F07BFD0123AB
:1036B00023712868042804D1002100F091FD012124
:1036C00004E00121042000F08BFD00211A2000F00D
:1036D00087FD70BD580A002010B5084C6379002B97
:1036E00005D00021052000F05DFD00236371052059
:1036F00000F08CFD43425841800010BD580A002064
:1037000010B5084CE37A002B05D000210B2000F007
:1037100049FD0023E3720B2000F078FD434258413D
:10372000800010BD580A0020E12110B5490204486C
:1037300000F057FEFFF7EAFEFFF7DAFE10BDC046C5
:103740005C0B0020F8B50B4E070030000D0000F0B8
:1037500087FE041EAC4200DD2C003D00EB1B9C42AA
:1037600005DD300000F086FE28700135F6E7200008
:10377000F8BDC0465C0B002010B50100014800F008
:1037800037FE10BD5C0B002010B51B20FEF7ECFAD5
:1037900010BD0420704710B51B20FEF7E5FA01208C
:1037A00010BD000010B501210D20FFF7DDFE012145
:1037B0000E20FFF7D9FE00210F20FFF7D5FE044CA5
:1037C000200000F09FF91021200000F0B7F910BD93
:1037D0008C0A002010B504680D20E30703D564109F
:1037E000FF2C03D91720FEF7BFFA06E0FFF7DAFF38
:1037F000E1B2024800F0C4F9002010BD8C0A00209C
:1038000010B5FFF7CFFF0021034800F0B9F90123FD
:103810004000184310BDC0468C0A00200122094B0D
:103820001A60094A1368002BFCD00322074B1B685F
:10383000D8171040C01801238010063840001843E4
:103840007047C04600C0004000C1004008C50040AD
:10385000F7B501260468344205D04268324202D0EE
:103860008368334201D10D2005E0521064100092AC
:10387000802C03D91520FEF777FA23E0009A162052
:10388000FF2AF8D85B1001931720FF2BF3D80E4FB7
:103890000E4D3B68002B03D1280000F0F7F93E6085
:1038A000E1B2280000F080FA6B462800197800F099
:1038B000AEF96B462800197900F0A9F9280000F04C
:1038C000DDFA0020FEBDC0467C0A0020A00A0020D0
:1038D000F7B501260468344202D04168314201D173
:1038E0000D2005E04B1064100193802C03D91520A6
:1038F000FEF73AFA2EE0019B1620FF2BF8D8164F60
:10390000164D3B68002B03D1280000F0BFF93E6044
:10391000E4B22100280000F047FA6B46280019792C
:1039200000F075F90021280000F04AFA002801D0C3
:1039300040420CE001222100280000F030FA28006B
:1039400000F05BF90028FAD0280000F05BF90123B1
:1039500040001843FEBDC0467C0A0020A00A00209B
:10396000F8B5274B06001A681F00264C002A19D10B
:10397000254D2B68002B04D1200000F087F901238E
:103980002B601D21200000F00FFA2A21200000F0FA
:103990003EF90121200000F03AF9200000F06EFA13
:1039A00001233B601D21200000F0FEF9F1B2200050
:1039B00000F02DF90021200000F002FA03000020A1
:1039C00083421BD101221D21200000F0E8F92000D4
:1039D00000F013F90028FAD0200000F013F97F2836
:1039E00001DD0138FF3803007F3301DA7F204042D8
:1039F00064237F215843494200F096FFF8BDC0463A
:103A0000780A0020A00A00207C0A002010B50120BE
:103A1000FFF7A6FF01234000184310BD10B5032097
:103A2000FFF79EFF01234000184310BD10B505208D
:103A3000FFF796FF01234000184310BD10B5FFF7B4
:103A400073FEE120C000FEF709FA0448FEF734FFD8
:103A5000FEF710FDFEF79CFF10BDC046D3650000C9
:103A600010B5FEF787F910BD70B5002504AC2478B9
:103A70000573A94205D10A4B0A4A23210A4801F0DD
:103A80006BF801600949920052589B0002715B5823
:103A90008371A3005B58856043710223C37170BDBD
:103AA00035690000F868000043690000CC69000037
:103AB000037B002B04D143738373036101330373CE
:103AC000704700001FB50191A02100240068C900C3
:103AD000D2B24450012A07D0A24203D0032A05D112
:103AE000042202E0022200E006221343034A83502C
:103AF000034B019AC250012343501FBD54050000DF
:103B00002405000010B50400FFF7D2FFA1222368AE
:103B1000A179D20099506179064A20009950217903
:103B200004329950044B19685A689B68FFF7CAFF22
:103B300010BDC0460C050000800A00204BB2002BCF
:103B40000CDB80233F290CD81F290CD80F290CD857
:103B500007290CD803290CD81B060BE080239B04F3
:103B600008E0DB0406E01B0504E05B0502E09B05C2
:103B700000E0DB050168014A8B5070472405000016
:103B80000368074A99501A00FC32D1680029FCD01A
:103B9000A321C90058580023C0B2D3607047C04663
:103BA0001C05000007B58022074BD2051A600022D1
:103BB0009A6002321A710F230C3200930349023BC0
:103BC0000348FFF751FF07BD800A00200030004086
:103BD0008C0A0020F8B505000E0017000024BC4236
:103BE00008D02B68315D1B6828009847002801D059
:103BF0000134F4E72000F8BD704710B51C3000F028
:103C0000D5FB10BD10B51C3000F0C2FB10BD70B567
:103C1000437E0D00002B05D06430040000F0D5FB7E
:103C2000002801D0002004E02000290000F0A1FBC2
:103C3000012070BD10B51C3000F0BEFB10BD0000AF
:103C4000F7B50193FA23002504009B0083600D4B18
:103C50004560083303601C300F00160000F07EFB47
:103C60002000643000F07AFB074AB600B3582761A1
:103C70006375019B20009B009B586576A576A37514
:103C8000FEBDC046AC690000CC6900000123A02243
:103C9000C375837D0C49C133FF33D2059B00995016
:103CA000437DC133FF339B009950CC210369074A00
:103CB000490499500521243A9950817D0832995040
:103CC000417D034A995070470C060000240500000E
:103CD0000C050000F7B5050000200C00019382429E
:103CE0005CD0161E402E00D940262F001C3738000D
:103CF00000F04AFBB1222B69D20080219C500122A6
:103D000089005A50A97E002901D11A621A60002444
:103D1000731E2A69A34206D1019B002B03D0802386
:103D200002219B00D150012313621300FC33D96898
:103D3000002902D1996A0029F9D0996A00290AD18B
:103D4000D960A323DB00D1583800C9B2013400F098
:103D500010FBA642DCD8019A2B69002A04D11A0074
:103D6000FC32916A00290AD001210022AA76596109
:103D70001900FC3188680028FCD08A6007E0012126
:103D8000A976D961D16C0029FCD00021D164FC3323
:103D90009A6A002A01D000229A62E0B2FEBD10B5F4
:103DA0000123FFF797FF10BD0300AC3310B50400EB
:103DB0001970643000F0E8FA0123637610BD00004A
:103DC000F8B500220D0001004276AC310369040011
:103DD0000878B121C9005850802189005A50013219
:103DE0001A629A6026006436300000F0DFFA00287C
:103DF0000ED03000276900F0CBFA1E4BF850236933
:103E0000FC331A6A002A0CD19A6A002AF9D008E019
:103E10002369002D0AD11A00FC32916A002905D1CC
:103E20000EE09A6A002AF3D11A62DBE701225A6196
:103E30001A00FC3291680029FCD00021916006E054
:103E40000121D961D16C0029FCD00021D1641A0074
:103E50000020FC32916A81420BD0074990625A5887
:103E600002305A50824204D0043A53425341023045
:103E7000C01AF8BD1C050000C404000010B50121E3
:103E8000FFF79EFF10BD000010B513231422024956
:103E90000248FFF7D5FE10BD00400040A00A0020F8
:103EA00003210A4802680A430260094802680A437B
:103EB00002600849084A094B9B1A03DD043BC858B5
:103EC000D050FBDC00F0B4F9FCF754F924050040B5
:103ED00054050040646C000000000020D400002065
:103EE000FEE7FEE7FEE7FEE7FEE7FEE7014B1860B0
:103EF0007047C04610000020F7B50023202877D86F
:103F00003C4B8000C258042A14D006D8022A0DD097
:103F10000ED80423012A14D069E0062A0ED00BD350
:103F20001A2A0DD002231B2A0BD060E0082308E0D8
:103F3000102306E0202304E0402302E0802300E079
:103F400001232D4A1268082A04D9092A05D00A211A
:103F5000022404E00821002401E011000124A0252E
:103F600001261C272548ED004651254D254E2D687C
:103F70001B02AD003D400195234D2D6800958559EC
:103F8000AC466746214D3D401D4385518359C025B0
:103F90009C46009BAD021D40FF2367461B023B4031
:103FA0002B43019D1D43009B5F0160231F402B009D
:103FB0003B431C4301238451154C036063680F4845
:103FC000002BFBD00024124B01255C60A123DB00F9
:103FD000C3584560A025ED0044511BB2914207D063
:103FE00002D98A1AD34003E0521A934000E000231A
:103FF0001800FEBDCC6900001400002000700040D5
:104000000C0000200405000008000020FF00FFFF56
:10401000FC700040F0B520286CD8374B8000C258A7
:10402000364B1E68002E2ED1C2243548A4000759F5
:10403000344B03253B40C0273F023B4303518023C1
:10404000893C9B00FF3C03512F4F03602F4B803C6A
:10405000D859FF3CA043D8510437D859A84320432E
:10406000D8510837D8590C35A843083D2843D851B2
:10407000A820C0001E508026C120760280001E505D
:104080001C601E4B1C6000231426214834005C4336
:10409000255804006F1C0FD1142058432250A02033
:1040A0000325C132FF329200C0051550194A08009D
:1040B0001268082A03D10BE0AA4218D1ECE7082ABB
:1040C00002D9083AD14002E00820821A9140080043
:1040D00014225343E3189A680C495132FF3292007C
:1040E00058605050DA68C1239B00CA5002E0013387
:1040F000032BCBD1F0BDC046CC690000580B00208B
:1041000000E100E0FF00FFFF040500000090004018
:1041100018000020100000201E4BF0B5596C18004C
:104120001D4A002914D0A025A12600230124ED0555
:10413000F600D1584F1C06D0D7187F68002F02D048
:1041400027008F40AF5114333C2BF2D1002343643E
:10415000131DA02540329446002001240F4EED058A
:10416000DA680F49920057180A495218526C002A0F
:104170000CD01A1F1268511C05D01968FF2902D0F3
:1041800021009140A9513A00FC32506414339C45FF
:10419000E6D1F0BDFC900040180000200C050000A6
:1041A0000090004000B5202816D80C4A83009B5888
:1041B000032911D8A0220800C133FF33D2059B0088
:1041C00000F014FB02080406002104E00C2102E0C8
:1041D000042100E00321D15000BDC046CC6900009D
:1041E00020280DD8074B8000C058A0220123D205FB
:1041F0008340002901D1044901E0A121C9005350A5
:104200007047C046CC6900000C0500000300002088
:10421000202B0AD8A222A021D200C9058858034A1F
:104220009B009B58D840012318407047CC69000080
:104230002D4B10B51A78012A19D12C4A1268120791
:1042400015D12B4AE0241168F022080010402142C9
:104250000BD128490968114209D12749274A116021
:104260008021274A0902116001E03028F1D01A7834
:10427000012A0DD11D490968090709D1F0201C49FF
:1042800009680140402903D11A490968014223D035
:104290001B68DBB2012B25D1144B1B681B0721D1F6
:1042A000134B1A68F0231A40A02A04D1114A12684D
:1042B0001A4203D016E0D02A14D1F7E7114B1A683E
:1042C000012A03D1C022104B1A600BE00F4A1A607A
:1042D0001A68012AFCD1F5E7C1218020C900C00578
:1042E0004250D5E710BDC046E00F00F0E40F00F0EB
:1042F000E80F00F0EC0F00F0DFFF07C004050040FE
:10430000186C004000EC064014EC06407593000069
:10431000F7B506000D000C008B180193019B671B7D
:104320009C4207D0336821781B68300098470134DD
:104330000028F3D13800FEBD70B505000C00081E42
:1043400007D001F0B5F82B6802005B682100280057
:10435000984770BD10B5FFF7EFFF10BD10B54022B4
:104360000021040000F081FC00232000236463642A
:1043700010BD3F23026C10B5541C2340446C9C427A
:1043800001D08154036410BD00230364436470476B
:10439000436C026C934206D03F21C25C01330B4058
:1043A0004364100001E0012040427047036C406C00
:1043B000181A00D540307047436C026C934201D00C
:1043C000C05C01E0012040427047036C406C5A1C05
:1043D0003F231340181A42424241D0B27047012095
:1043E000704710B503681322DB69984710BD70470A
:1043F0000369054A9950FC331A6A002AFCD000224E
:1044000001201A627047C0461C050000030010B569
:104410005C331A781F2313400122110099400D4B81
:104420000424D967C221036989005C505A60DA60AC
:10443000A0220021D20099500122074952425A502D
:10444000064914305A500C395A5008315A50FFF767
:104450009BFF10BD04E100E00C0500001405000006
:1044600010B51430FFF7A2FF10BD10B51430FFF7E0
:10447000A3FF10BD10B51430FFF78AFF10BD000078
:10448000030070B55E331C780269604BD4500300A2
:104490005D331C785E4BD450030061331C785D4B58
:1044A000012C0CD105005F352E78A225ED00565168
:1044B000050060352E78A125ED00565100E000245E
:1044C000D4509623DB00994238D996231B01994298
:1044D00037D996235B01994236D996239B0199429D
:1044E00034D9E1239B01994232D99623DB019942C9
:1044F00031D9E123DB0199422FD996231B0299423E
:104500002DD9E1231B0299422BD996235B029942B4
:1045100029D9E1235B02994227D9E1239B029942E1
:1045200025D93D4B994224D9E123DB02994223D975
:10453000E1231B03994221D8384B21E09E23DB0263
:104540001EE09D231B031BE0354B19E0354B17E0A4
:10455000EC239B0314E0344B12E0344B10E0344B5B
:104560000EE0344B0CE0344B0AE0344B08E0344BA3
:1045700006E08023DB0403E0324B01E080235B058F
:104580003149002453500423243953501100FC3185
:10459000CC600C62C1210134890014605C309460ED
:1045A000535003781F202200D9B208408240803443
:1045B0002648FF345BB20251002B13DA0F230B4065
:1045C000083B234C9B089B001B1903242140A1405E
:1045D000FC348C40DD69A543C0248C402100294374
:1045E000D96111E0194C9B089B001B190324214041
:1045F000A140C025FC348C40AD005E59A643C024C8
:104600008C40210031435951026070BD0C050000FF
:10461000140500006C05000090D0030000D0BE0E11
:1046200000B013000050270000A04E0000F07500FD
:1046300000509D0000F0EB0000903A0100E0D7012F
:1046400000B0AF0300705F072405000000E100E048
:1046500000ED00E0F7B5009308AB1B78002501934F
:10466000FA2304009B0083600E4B4560083303600F
:1046700014300F001600FFF771FE23005C33276132
:104680001E70009B084A9B00995823005D331970E7
:10469000019B20009B009A5823005E33DD701A7046
:1046A000FEBDC046506A0000CC690000036910B529
:1046B0001A00FC32D2680400002A0AD0A322D200D9
:1046C00099581430C9B2FFF754FE00222369FC3315
:1046D000DA6010BD10B50248FFF7E8FF10BDC04614
:1046E0005C0B0020162307B5022200930249013B10
:1046F0000248FFF7AFFF07BD002000405C0B002021
:104700007047000010B500F047F8FFF7F9FF0120EF
:1047100000F024F8FFF792F9FFF7A2F9024B002B03
:10472000FAD000E000BFF7E700000000084A09499E
:10473000094B10B51B688858FA22190A1B06184342
:104740009200002300F0DCF94904C00B084310BDBF
:104750000405000000100140C00B002070B5041ECD
:1047600009D0FFF7E3FF050000F014F8FFF7DEFFC4
:10477000401B8442F8D870BD0022044B9A60044A62
:1047800013680133DBB213607047C046FC10014070
:10479000C00B002070470000C421114A8900505806
:1047A000104B0340C0200002034353508023913933
:1047B0009B02FF39535013608023A3220021DB05A5
:1047C000D20099500122A1209A60074BC0001950D5
:1047D000C120023180001950403019501A607047D2
:1047E00000E100E0FF00FFFF0010014002B471464D
:1047F00049084900095C49008E4402BC7047C04624
:1048000003B47146490840004900095A49008E44E2
:1048100003BC7047002243088B4274D303098B42C8
:104820005FD3030A8B4244D3030B8B4228D3030C80
:104830008B420DD3FF22090212BA030C8B4202D322
:104840001212090265D0030B8B4219D300E0090A4A
:10485000C30B8B4201D3CB03C01A5241830B8B4253
:1048600001D38B03C01A5241430B8B4201D34B033C
:10487000C01A5241030B8B4201D30B03C01A5241A1
:10488000C30A8B4201D3CB02C01A5241830A8B4226
:1048900001D38B02C01A5241430A8B4201D34B020F
:1048A000C01A5241030A8B4201D30B02C01A524173
:1048B000CDD2C3098B4201D3CB01C01A5241830927
:1048C0008B4201D38B01C01A524143098B4201D361
:1048D0004B01C01A524103098B4201D30B01C01A8C
:1048E0005241C3088B4201D3CB00C01A5241830806
:1048F0008B4201D38B00C01A524143088B4201D333
:104900004B00C01A5241411A00D201465241104692
:104910007047FFE701B5002000F0F0F802BDC04687
:104920000029F7D076E7704703460B437FD4002277
:1049300043088B4274D303098B425FD3030A8B4233
:1049400044D3030B8B4228D3030C8B420DD3FF229D
:10495000090212BA030C8B4202D31212090265D06B
:10496000030B8B4219D300E0090AC30B8B4201D31E
:10497000CB03C01A5241830B8B4201D38B03C01A65
:104980005241430B8B4201D34B03C01A5241030BDC
:104990008B4201D30B03C01A5241C30A8B4201D38D
:1049A000CB02C01A5241830A8B4201D38B02C01A38
:1049B0005241430A8B4201D34B02C01A5241030AAF
:1049C0008B4201D30B02C01A5241CDD2C3098B4294
:1049D00001D3CB01C01A524183098B4201D38B0111
:1049E000C01A524143098B4201D34B01C01A5241B4
:1049F00003098B4201D30B01C01A5241C3088B42F9
:104A000001D3CB00C01A524183088B4201D38B00E3
:104A1000C01A524143088B4201D34B00C01A524185
:104A2000411A00D201465241104670475DE0CA0F5C
:104A300000D04942031000D34042534000229C461C
:104A400003098B422DD3030A8B4212D3FC22890126
:104A500012BA030A8B420CD3890192118B4208D3FC
:104A6000890192118B4204D389013AD0921100E05E
:104A70008909C3098B4201D3CB01C01A5241830972
:104A80008B4201D38B01C01A524143098B4201D39F
:104A90004B01C01A524103098B4201D30B01C01ACA
:104AA0005241C3088B4201D3CB00C01A5241830844
:104AB0008B4201D38B00C01A5241D9D243088B429A
:104AC00001D34B00C01A5241411A00D2014663463D
:104AD00052415B10104601D34042002B00D54942A1
:104AE000704763465B1000D3404201B5002000F0E0
:104AF00005F802BD0029F8D016E770477047C04698
:104B0000F0B54F464646C0B41604360C99463300FD
:104B100005042C0C070C150C63437E436F4365435F
:104B20001C0CAD1964199C46A64203D980235B0274
:104B3000984647446346250CEF191D044B464A43EB
:104B400043432D0C240464199918C91920000CBC86
:104B500090469946F0BDC0467FB51D000A4B060041
:104B60001B68D868002A02D1084C230001E013001A
:104B7000074C0293009133002A000649019400F08B
:104B800021F800F007FEC046B40000200C650000CC
:104B9000806A00008D6A0000084B10B50400002BED
:104BA00002D0002100E000BF054B1868836A002B8B
:104BB00000D09847200001F0D7FAC046000000005E
:104BC000C06A00000EB403B5010003AB044804CB77
:104BD0000068019300F016F902B008BC03B0184752
:104BE000B40000200E4B70B500251E000D4CE41AD9
:104BF000A410A54204D0AB00F35898470135F8E75C
:104C000001F0B4FA084B00251E00084CE41AA41069
:104C1000A54204D0AB00F35898470135F8E770BDC2
:104C2000BC000020BC000020BC000020CC00002004
:104C300010B5034B0100186800F066F810BDC046BF
:104C4000B400002010B5034B0100186800F016F8FE
:104C500010BDC046B4000020002310B59A4203D016
:104C6000CC5CC4540133F9E710BD030082189342B1
:104C700002D019700133FAE77047000030B50029FF
:104C80003ED004390B68002B00DAC9181D4A13689E
:104C90001400002B02D14B60116031E08B420DD922
:104CA0000A688818834203D118685B6882180A6012
:104CB0004B60216024E08A4203D813005A68002A1E
:104CC000F9D11D685C198C420BD109686918581814
:104CD0001960824214D110685268411819605A60F4
:104CE0000EE08C4202D90C23036009E008680C181E
:104CF000A24203D114685268201808604A605960C3
:104D000030BDC046C80B0020032370B5CD1C9D43A9
:104D1000083506000C2D01D20C2505E0002D03DA24
:104D20000C230020336040E0A942F9D81F4B1C68D7
:104D30001A002100002913D00B685B1B0DD40B2B2C
:104D400002D90B60CC181EE08C4202D1636813605C
:104D50001AE04B6863600C0016E00C004968E9E754
:104D6000134C2368002B03D1300000F033FB20608C
:104D70002900300000F02EFB431CD1D00323C41CBB
:104D80009C43A0420AD12560200007220B30231D3E
:104D90009043C31A09D05A42E25006E0211A30006B
:104DA00000F018FB431CEED1BAE770BDC80B002021
:104DB000C40B0020936810B5013B9360002B05DA0B
:104DC0009469A34208DBCBB20A2B05D01368581CA8
:104DD00010601970C8B201E000F010FC10BDF8B509
:104DE00006000F001400D518AC4208D021783A0014
:104DF0003000FFF7DFFF0134431CF5D100E0002055
:104E0000F8BD0000F0B59FB006000F0002920593B8
:104E1000002804D08369002B01D100F0B7FD7F4B3F
:104E20009F4201D1776808E07D4B9F4201D1B7686E
:104E300003E07C4B9F4200D1F768BB891B070AD572
:104E40003B69002B07D0002306AD6B6120336B76E6
:104E50001033AB763DE03900300000F027FC00282D
:104E6000F1D001204042D6E0059A111D126805914B
:104E7000002A00DA7FE00992013423782E2B00D13A
:104E80008DE021780322684800F066FE002807D0F4
:104E9000654B2A68C01A4023834013432B600134BA
:104EA0002178631C062261480293297600F054FEA3
:104EB000002800D19DE05E4B002B00D090E007223F
:104EC000059B07339343083305936B69039A9B183B
:104ED0006B61029C2378002B04D1029BE31A04939C
:104EE00012D003E0252BF8D00134F3E7049B029A9B
:104EF00039003000FFF773FF431C00D186E06A6978
:104F0000049B944663446B612378002B7ED001227E
:104F1000002352426A6002A95432521801342B60B5
:104F2000EB60AB601370AB6521780522414800F05F
:104F300013FE002808D03F4B2A68C01A0123834083
:104F400013432B600134EFE72B68DA0604D55322B4
:104F5000202102A8121811701A0704D553222B2100
:104F600002A81218117022782A2A00D17CE7099B26
:104F700000200A2105E05242EA60022213432B601E
:104F80007AE72278303A092A04D84B4301349B1837
:104F90000120F6E7002800D16FE709936DE76378F9
:104FA0002A2B0AD1059B02341A1D1B680592002B7F
:104FB00001DA01235B42079363E700230A201A000A
:104FC00001346B6021783039092904D84243013417
:104FD00052180123F6E7002B00D152E7079250E761
:104FE00005AB00933A00144B2900300000E000BFED
:104FF00007E005AB00933A000F4B2900300000F0AA
:105000008BF80390039B013300D05EE7BB895B06FE
:1050100000D526E70B981FB0F0BDC046F86B000026
:10502000186C0000386C0000CA6A0000CE6A0000EC
:1050300000000000C46A0000DF4D0000F7B5170053
:1050400001938A680B6900900C00934200DA130008
:1050500022003B6043321278002A01D001333B60CA
:1050600023689B0602D53B6802333B600625236814
:105070001D401ED0230043331B785A1E93412268E3
:1050800092061CD53020E1184331087021005A1CCB
:1050900045310978A2184332023311700FE0220023
:1050A0000123193201990098089EB047431C0ED085
:1050B0000135E3683A689B1A9D42F0DBDAE722008B
:1050C000019943320098089DA847431C02D1012052
:1050D000404220E006232068E1683A68034000254A
:1050E000042B03D18D1AEB43DB171D40A368226903
:1050F000934201DD9B1AED180027BD420AD0220021
:1051000001231A3201990098089EB047431CDED053
:105110000137F2E70020FEBDF0B58BB006920A0021
:1051200043320793059004920A7E0C00109B6E2A6E
:1051300000D1ABE011D8632A22D009D8002A00D1CF
:10514000B5E0582A00D0C5E045310A70814A4FE0E9
:10515000642A1DD0692A1BD0BCE0732A00D1AAE0C2
:1051600009D86F2A29D0702A00D0B3E0202209681C
:105170000A43226037E0752A1FD0782A33D0A9E08D
:105180000E001A684236111D196013683370A4E0CE
:1051900021681A68080606D4490604D5111D19604D
:1051A0000023D55E02E0111D19601568002D3BDA61
:1051B0002D23049A6D42137036E021681A680806A0
:1051C00006D4490604D51568111D1960ADB202E078
:1051D000111D196015685F4B227E039308276F2A03
:1051E0001DD00A271BE022007821453211705A4A4F
:1051F00019680392081D226818600D68100602D411
:10520000500600D5ADB2D30702D520231A43226041
:105210001027002D03D1202322689A432260230007
:10522000002243331A7002E00A274A4B0393636853
:10523000A360002B09DB0422216891432160002D2B
:1052400005D1049E002B11D07BE0002D79D0049E67
:1052500028003900FFF764FB039B013E5B5C2800DC
:1052600033703900FFF7D6FA051EF1D1082F09D1A6
:105270002368DB0706D563682269934202DC30238A
:10528000013E3370049B9B1B23612BE009681A6865
:10529000080607D4490605D5111D19601368A28AAE
:1052A0001A8004E0111D1960136862691A600023F6
:1052B000049E236116E01A68111D1960166800210A
:1052C0006268300000F048FC002801D0801B60605C
:1052D000636803E026004236327001232361002315
:1052E000049A1370079B09AA00932100069B059856
:1052F000FFF7A4FE431C02D10120404227E02369AE
:10530000320006990598079DA847431CF4D02368EE
:1053100000259B070FD4099BE068984217DA180014
:1053200015E022000123193206990598079EB0471F
:10533000431CE1D00135E368099A9B1A9D42F0DBDA
:10534000E9E72600039B42361B7833708EE70BB0EB
:10535000F0BDC046D56A0000E66A0000154B10B5E6
:105360001C68A36B002B15D11820FFF761FC124BB2
:10537000A0630380114B01224380114B8380114BAA
:10538000C380114B038105234381063383810023AE
:1053900002614361A46B0D4A206961690C4BFFF700
:1053A000AFFB012200238018594120616161480050
:1053B000400810BDB40000200E330000CDABFFFF4D
:1053C000341200006DE6FFFFECDEFFFF2D7F954CF1
:1053D0002DF45158002370B5064C050008002360D9
:1053E00000F0ACFE431C03D12368002B00D02B60DF
:1053F00070BDC046E81E00200CB430B5164B9DB001
:105400000C1E1D6804DA8B2301202B6040421DE036
:10541000822302A99B008B810023029008619C4299
:1054200000D0631E8B604B6101235B42CB81209ACD
:1054300021AB2800019300F037FC431C01DA8B23D9
:105440002B60002C02D00023029A13701DB030BCD8
:1054500008BC02B01847C046B40000200EB410B516
:105460009DB002A9029008610B48822488604861BF
:10547000012040421FABC881084804CBA40000684B
:1054800001938C8100F010FC0023029A13701DB070
:1054900010BC08BC03B01847FFFFFF7FB40000201A
:1054A000031C0A7801311A700133002AF9D17047C0
:1054B0000023C25C0133002AFBD1581E7047000054
:1054C000F0B51E00454B87B01B680192029308227D
:1054D0000B00059003911C7802995D1C091948780E
:1054E000104001D02B00F6E72D2C04D19D1C5C78D8
:1054F0000123009304E000902B2C01D15C789D1CCB
:10550000002E02D0102E0AD162E0302C5ED1202273
:105510002B789343582B54D110266C780235009F7A
:1055200031007B1E9F412E4BFF183800FFF7F8F922
:10553000380004913100FFF76DF9002303220700C2
:1055400094461800029A121951780422114201D08F
:10555000303C07E06246114017D03722012900D0C5
:105560002032A41AA64210DD5A1C0BD0B84207D82C
:1055700002D1049B9C4203DC70430123201801E00C
:1055800001235B422C780135DCE75A1C0BD10098D3
:10559000059A431E9841124BC01822231360019BA9
:1055A000002B0AD117E0009A002A00D04042019A4D
:1055B000002A10D0039A002B00D06A1E019B1A60AB
:1055C00009E03024002EAAD10826A8E70A26A6E77B
:1055D000302C9CD0A3E707B0F0BDC046B800002037
:1055E000FFFFFF7F10B513000A00010002480068AA
:1055F000FFF766FF10BDC046B4000020F8B50500F7
:105600000F001400002804D08369002B01D100F0A2
:10561000BDF9234B9C4201D16C6808E0214B9C42B0
:1056200001D1AC6803E0204B9C4200D1EC68A36937
:10563000A360A3891B070AD52369002B07D0236821
:105640002269FEB2981A636998420FDB08E02100D4
:10565000280000F02BF80028F1D0012040421DE086
:105660002100280000F024F90028F6D1A3680130B9
:10567000013BA36023685A1C22601F706369984233
:1056800005D0A3893000DB0708D50A2E06D12100FA
:10569000280000F00DF90028DFD13000F8BDC04629
:1056A000F86B0000186C0000386C0000354B70B5CA
:1056B0001D6806000C00002D05D0AB69002B02D13F
:1056C000280000F063F9304B9C4201D16C6808E07F
:1056D0002E4B9C4201D1AC6803E02D4B9C4200D183
:1056E000EC68A3899AB2110723D4D10607D4092202
:1056F0000120326037321343A381404240E0530718
:1057000013D5616B002908D023004433994202D09D
:105710003000FFF7B3FA002363632422A389934385
:10572000A38100236360236923600822A3891343B4
:10573000A3812369002B0BD1A023A2899B001340D6
:1057400080229200934203D02100300000F0B2F991
:105750000123A289134005D00023A36063695B4243
:10576000A36103E0910700D46369A360002023696B
:10577000834205D1130603D540231A43A281013881
:1057800070BDC046B4000020F86B0000186C00002B
:10579000386C000010B5062000F0AEFB012000F0D0
:1057A000E3FC0000F7B58A8905000C0013075AD402
:1057B0004B68002B02DC0B6C002B19DDE76A002F15
:1057C00016D000232E682B6080235B011A4001D085
:1057D000606D14E00123216A2800B847431C0ED1F4
:1057E0002B68002B0BD01D2B01D0162B02D12E6065
:1057F00000205AE04022A3891343A38155E0A389E6
:105800005B0706D56368C01A636B002B01D0236C5D
:10581000C01A00230200216A2800E76AB847A3895A
:10582000421C06D129681D293AD8204ACA40D2070D
:1058300036D50022626022692260DB0405D5431C54
:1058400002D12B68002B00D16065616B2E600029AE
:10585000CED023004433994202D02800FFF70EFA3D
:105860000020606321E00F69002FC1D00B680F603A
:10587000DB1B01930023920700D14B69A36003E077
:10588000019B3F181B1A0193019B002BB0DD019B6C
:105890003A00216A2800A66AB0470028F0DCA389F4
:1058A000402201201343A3814042FEBD010040205D
:1058B0000B6970B505000C00002B01D100201CE025
:1058C000002804D08369002B01D100F05FF80B4B56
:1058D0009C4201D16C6808E0094B9C4201D1AC6844
:1058E00003E0084B9C4200D1EC680C22A35E002B25
:1058F000E4D021002800FFF755FF70BDF86B0000D1
:10590000186C0000386C000010B5024900F0B0F8C7
:1059100010BDC046B1580000002310B5040003605C
:105920004360836081814366C28103614361836117
:10593000190008225C30FFF798F9054B2462636276
:10594000044BA362044BE362044B236310BDC046C7
:10595000395F0000615F0000995F0000C55F0000D3
:1059600070B568254B1E5D430E0029007431FFF7AA
:10597000CBF9041E08D000212A00016046600C30DB
:10598000A0606832FFF771F9200070BD836913B51C
:105990000400002B28D18364C3640365134B144AAD
:1059A0001B6882620193984201D101238361200028
:1059B00000F020F86060200000F01CF8A0602000DB
:1059C00000F018F80022E06004216068FFF7A4FFEF
:1059D00001220921A068FFF79FFF02221221E0683F
:1059E000FFF79AFF0123A36113BDC046C06A000000
:1059F00009590000F8B51D4B06001D68AB69002B66
:105A000002D12800FFF7C2FF4835AC686B68013B44
:105A100005D40C22A75E002F10D06834F7E72B685E
:105A2000002B01D02D68F0E704213000FFF798FF2C
:105A300028600028F6D10C23336016E001232000F3
:105A40005B42E3810233A38167662760A7606760DA
:105A500027616761A7615C3008223900FFF705F90B
:105A600020006763A763A764E764F8BDC06A00000D
:105A7000F7B504000700002601914834002C16D029
:105A80006368A5680093009B013B00930DD4AB892C
:105A9000012B08D90E22AB5E013304D02900380057
:105AA000019B984706436835EDE72468E6E7300038
:105AB000FEBD0000F0B58B8991B006000C009B077D
:105AC00026D40E23C95E002904DA8023A5891D404F
:105AD00010D10CE001AA00F0A1FA0028F5DBF023B8
:105AE000029D1B021D401A4BED186B425D41802741
:105AF000FF0001E00025402739003000FFF704F9DE
:105B000000280CD1A3899A051FD402221343A38134
:105B100023004733236023610123636115E0802262
:105B20000C4BB362A38920601343A381206167619A
:105B3000002D0AD00E23E15E300000F081FA00282B
:105B400003D00122A3891343A38111B0F0BDC04645
:105B500000E0FFFF09590000C9B28218904204D04A
:105B600003788B4202D00130F8E70020704710B56F
:105B7000884202D98B18984201D3002305E09B1A72
:105B8000013A08D3995C8154FAE7934203D0CC5C84
:105B9000C4540133F9E710BDF8B506000C00150038
:105BA000002904D11100FFF7AFF8040018E0002A23
:105BB00003D1FFF763F82C0012E000F067FA85428A
:105BC0000ED929003000FFF79FF8071E07D02100EB
:105BD0002A00FFF741F821003000FFF74FF83C00A2
:105BE0002000F8BDF0B58E6885B007000C00039268
:105BF00001939E4243D890238A89DB001A423ED00B
:105C000003250969236801985B1A029363695D4360
:105C1000EB0F5D19029B6D1001331B18AB4200D9CD
:105C20001D00530510D529003800FFF76DF8061E3A
:105C300014D0029A2169FFF70FF8A289194B13407B
:105C400080221343A38112E02A003800FFF7A4FF4B
:105C5000061E0CD121693800FFF710F80C234022F2
:105C600001203B60A38940421343A38117E0029BBC
:105C70002661F61826606561019EED1AA560019BFC
:105C8000B34200D21E00320003992068FFF76FFF75
:105C90000020A3689B1BA36023689E19266005B0A3
:105CA000F0BDC0467FFBFFFFF0B59FB002900593AB
:105CB0008B890F0016001B0610D50B69002B0DD128
:105CC0004021FFF721F838603861002804D10C2307
:105CD000029A01381360D8E040237B61002306ADAF
:105CE0006B6120336B761033AB7634002378002B56
:105CF00003D1A31B049312D003E0252BF9D0013468
:105D0000F4E7A31B320039000298FFF76BFF431C36
:105D100000D1B4E06A69049B944663446B612378C4
:105D2000002B00D1ABE00122002352426A6002A99D
:105D30005432521801342B60EB60AB601370AB65CA
:105D4000534E217805223000FFF706FF002807D0C8
:105D50000123801B83402A68013413432B60EFE743
:105D60002B68DA0604D55322202102A812181170DC
:105D70001A0704D553222B2102A812181170227879
:105D80002A2A03D0099B00200A210EE0059A111D42
:105D900012680591002A01DB099204E05242EA6090
:105DA000022213432B6001340BE02278303A092A97
:105DB00004D84B4301349B180120F6E7002800D09B
:105DC000099323782E2B1ED163782A2B0AD1059BA9
:105DD00002341A1D1B680592002B01DA01235B4275
:105DE000079310E000230A201A0001346B60217829
:105DF0003039092904D84243013452180123F6E707
:105E0000002B00D00792234E217803223000FFF7A9
:105E1000A3FE002806D04023801B83402A6801345B
:105E200013432B60217806221B48661C2976FFF756
:105E300093FE002812D0194B002B06D10722059B98
:105E4000073393430833059314E005AB00933A00FE
:105E5000134B2900029800E000BF07E005AB009358
:105E60003A000F4B29000298FFF756F90390039B65
:105E7000013304D06B69039A9B186B6135E7BB89CA
:105E80000B985B0601D5012040421FB0F0BDC04613
:105E9000C46A0000CA6A0000CE6A00000000000068
:105EA000E55B000070B504000D1E1F2D04D91623FC
:105EB0000360012040421EE0426C002A04D08B00A7
:105EC000D2181368002B08D1200000F031F82A0006
:105ED0000100200000F01AF80DE00020012B0AD08C
:105EE000591C03D117332360013004E0002428003B
:105EF00014609847200070BD10B5034B010018686E
:105F0000FFF7D0FF10BDC046B4000020002370B5DD
:105F1000064C050008001100236000F0F7F8431C50
:105F200003D12368002B00D02B6070BDE81E002039
:105F300010B500F0DBF810BD70B50C000E25495F00
:105F400000F0B0F8002803DB636D1B18636503E005
:105F5000A289024B1340A38170BDC046FFEFFFFF33
:105F6000F8B51F008B8905000C001600DB0505D570
:105F70000E23C95E0022022300F074F8A289054BAB
:105F800028001340A38132000E23E15E3B0000F0A5
:105F90001FF8F8BDFFEFFFFF70B50C000E25495F3D
:105FA00000F060F8A389421C03D1054A1340A38185
:105FB00004E0802252011343A381606570BDC04696
:105FC000FFEFFFFF10B50E23C95E00F015F810BDFE
:105FD00070B50500080011000022064C22601A006E
:105FE00000F0BAF8431C03D12368002B00D02B60CB
:105FF00070BDC046E81E0020002370B5064C0500A9
:106000000800236000F062F8431C03D12368002BD2
:1060100000D02B6070BDC046E81E0020002370B584
:10602000064C050008001100236000F057F8431CDF
:1060300003D12368002B00D02B6070BDE81E002028
:10604000002370B5064C05000800236000F056F8E8
:10605000431C03D12368002B00D02B6070BDC046C9
:10606000E81E002070B50500080011000022064C53
:1060700022601A0000F052F8431C03D12368002B61
:1060800000D02B6070BDC046E81E00200B1F1A68B0
:10609000101F002A04DA891804390B68D018043854
:1060A0007047000070B50500080011000022064C82
:1060B00022601A0000F03AF8431C03D12368002B39
:1060C00000D02B6070BDC046E81E00205822012081
:1060D000014B40421A607047E81E00205822012000
:1060E000014B40421A607047E81E002058220120F0
:1060F000014B40421A607047E81E00205822024BB4
:1061000000201A607047C046E81E00205822012077
:10611000014B40421A607047E81E002058220120BF
:10612000014B40421A607047E81E002058220120AF
:10613000014B40421A607047E81E0020044A136871
:10614000002B03D01818106018007047014BF9E7B6
:10615000CC0B0020F01E002058220120014B4042B1
:106160001A607047E81E0020FEE7C046F8B5C0463A
:10617000F8BC08BC9E467047F8B5C046F8BC08BCE1
:106180009E467047AE06000040060000BE060000B6
:10619000F4060000300700006A070000A6070000B0
:1061A000D20700001008000056080000B2080000E6
:1061B000F808000066090000B4090000E0090000CA
:1061C0001A0A0000640A00008C0A0000C40A0000D9
:1061D000FC0A0000380B0000BE0B0000860C00001B
:1061E000F40C0000300D0000720D0000940D000052
:1061F0009C0D00007C0E0000AE060000AE06000004
:10620000AE060000AE060000AE060000AE060000BE
:10621000C80E0000120F0000600F0000E60F000023
:1062200082100000D01000001A1100006011000060
:10623000AC110000F81100004412000090120000A0
:10624000DC1200001A13000086130000B6130000D1
:106250000C14000058140000A4140000DE14000008
:106260002A150000AE060000AE060000AE060000D3
:10627000AE06000076150000A6150000D615000039
:1062800002160000321600005E160000AE06000086
:10629000AE060000AE060000AE0600008E1600003E
:1062A000D616000022170000521700007E170000CB
:1062B000C4170000AE060000AE060000AE060000E7
:1062C000AE06000004180000341800006418000036
:1062D00094180000C0180000F01800001C190000FD
:1062E0004619000070190000A0190000D019000024
:1062F000FC190000281A0000581A0000841A000037
:10630000AE060000AE060000AE060000AE060000BD
:10631000AE060000B41A0000E01A00000C1B0000DA
:10632000381B0000741B0000A41B0000D41B0000DD
:10633000041C0000341C0000601C00008E1C0000C7
:10634000BE1C0000EC1C00002C1D0000AE0600006E
:10635000AE060000AE060000AE060000AE0600006D
:10636000AE060000AE060000AE060000AE0600005D
:10637000AE060000AE060000AE060000AE0600004D
:10638000AE06000066616C73650074727565006C22
:10639000697374206F66202564206974656D7300CD
:1063A0006F626A656374206F6620636C6173733A11
:1063B00020256400537461636B20756E646572669A
:1063C0006C6F77000D0A564D2050616E69633A205C
:1063D00025730D0A00496E73756666696369656E9B
:1063E00074206D656D6F727920666F72204D6963E0
:1063F000726F426C6F636B73206F626A65637420A7
:106400006865617000496E73756666696369656E7B
:1064100074206D656D6F727920666F72204D6963AF
:10642000726F426C6F636B7320737461636B006295
:106430006164206F626A65637420617420256C64F6
:106440000A0025783A20256420776F7264732C2027
:10645000636C61737349442025640A004865616474
:1064600065723A2025780A0009307825782C0A00D0
:1064700025642025642025642025640A0042616487
:10648000207265636F726420666F756E6420647538
:1064900072696E6720696E697469616C697A61748A
:1064A000696F6E210A004E6F7420656E6F756768A4
:1064B00020726F6F6D206576656E206166746572FF
:1064C00020636F6D70616374696F6E0A005265734B
:1064D000746F72696E6720256420736372697074CB
:1064E000732E2E2E0053746172746564002D2D2D51
:1064F0002D2D0A0050657273697374656E74204D9A
:10650000656D6F727920546573740A0A000A496ECA
:10651000697469616C697A696E67204D656D6F7227
:10652000790A004D656D6F727920696E74697469BE
:10653000616C697A65643B2077726974696E672063
:106540007265636F7264732E2E2E0A005265636F3C
:106550007264206174206F66667365742025643AE6
:1065600020256420256420256420256420282564B6
:1065700020776F726473290A0046696E616C3A2055
:1065800063757272656E742025642075736564206E
:1065900025642063302025642063312025640A00AF
:1065A0004E6F2066726565207461736B20656E7432
:1065B0007269657300416C6C207461736B73207336
:1065C000746F70706564007630343100202573205C
:1065D00025730057656C636F6D6520746F204D697E
:1065E00063726F426C6F636B7321001A1B1C030490
:1065F0000607090A17181900000000000100000032
:10660000020000000300000004000000050000007C
:10661000060000000700000008000000090000005C
:106620000A0000000B0000000C0000000D0000003C
:106630000E0000000F00000010000000120000001B
:106640001400000016000000180000001A000000EE
:106650001C0000001E0000002000000023000000BD
:1066600026000000290000002C0000002F00000080
:1066700032000000360000003A0000003E0000003A
:1066800042000000460000004B00000050000000E7
:10669000550000005A000000610000006800000082
:1066A0006F000000760000007D0000008400000004
:1066B0008B0000009200000099000000A000000084
:1066C000A7000000AE000000B5000000BC00000004
:1066D000C3000000CA000000D1000000D800000084
:1066E000DF000000E6000000ED000000F400000004
:1066F000FB000000FF000000000000000008080888
:1067000000080A4A4000000A5FEA5FEA0ED92ED369
:106710006E19324489330C924C924D0808000000E7
:1067200004880808040804848488000A448A400015
:10673000048EC480000000048800000EC000000029
:1067400000080001224488100C9252524C048C84A0
:10675000848E1C824C901E1EC244924C06CA525F0C
:10676000E21FF01EC13E02448ED12E1FE24488106B
:106770000ED12ED12E0ED12EC488000800080000A4
:10678000048004880244880482000EC00EC00804FD
:106790008244880ED126C0040ED135B36C0C925EB3
:1067A000D2521C925C925C0ED010100E1C9252526F
:1067B0005C1ED01C901E1ED01C90100ED013712E8B
:1067C00012525ED2521C8808081C1FE242524C1220
:1067D00054981492101010101E113B75B1311139DC
:1067E00035B3710C9252524C1C925C90100C925228
:1067F0004C861C925C92510ED00C825C1FE4848407
:1068000084125252524C1131312A44113135BB712C
:1068100012524C9252112A4484841EC488101E0EB7
:10682000C808080E10080482410EC242424E048A73
:10683000400000000000001F0804800000000ED28D
:10684000524F10101C925C000ED0100E02424ED21D
:106850004E0C925C900E06C81C88080ED24EC24C9C
:1068600010101C92520800080808024002424C1006
:10687000149814920808080806001B75B131001C12
:10688000925252000C92524C001C925C90000ED21C
:106890004EC2000ED010100006C8049808080EC89A
:1068A00007001252524F0011312A4400113135BBFA
:1068B00000124C8C9200112A4498001EC4881E06B7
:1068C000C48C8486080808080818080C881800007A
:1068D0000C83606D6963726F3A6269740000000036
:1068E00000000000010000000200000003000000A2
:1068F000040000000A000000535049436C617373A8
:106900003A3A535049436C617373284E52465F5371
:1069100050495F547970652A2C2075696E74385F10
:10692000742C2075696E74385F742C2075696E74D0
:10693000385F742900705F73706920213D204E55C7
:106940004C4C002F55736572732F6A6F686E6D61C2
:106950006C6F6E65792F4C6962726172792F41722A
:106960006475696E6F31352F7061636B6167657334
:106970002F73616E646565706D69737472792F68C9
:10698000617264776172652F6E5246352F302E34F6
:106990002E302F6C69627261726965732F53504992
:1069A0002F5350492E63707000000000000000005B
:1069B000000000000F3C0000D53B0000FB3B000046
:1069C000053C0000353C0000F93B000003000000DE
:1069D00002000000010000000400000005000000AB
:1069E000110000000C0000000B000000120000006D
:1069F0000A000000060000001A0000001400000059
:106A00001700000016000000150000001000000034
:106A1000FFFFFFFFFFFFFFFF000000001E00000060
:106A20001900000018000000070000000800000026
:106A3000090000000D0000000E0000000F00000023
:106A40001C0000001B0000001D00000013000000DF
:106A50000000000000000000F143000011430000AE
:106A600061440000754400006B440000EF430000E7
:106A7000E3430000814400000D440000DF430000B8
:106A80002C2066756E6374696F6E3A2000617373B3
:106A9000657274696F6E2022257322206661696CAD
:106AA00065643A2066696C6520222573222C206C6F
:106AB000696E65202564257325730A004300000074
:106AC00054000020232D302B2000686C4C0065669C
:106AD000674546470030313233343536373839412F
:106AE0004243444546003031323334353637383945
:106AF0006162636465660000202020202020202041
:106B0000202828282828202020202020202020205D
:106B1000202020202020202088101010101010107D
:106B200010101010101010100404040404040404C5
:106B30000404101010101010104141414141410156
:106B40000101010101010101010101010101010135
:106B50000101011010101010104242424242420244
:106B60000202020202020202020202020202020205
:106B700002020210101010200000000000000000AF
:106B80000000000000000000000000000000000005
:106B900000000000000000000000000000000000F5
:106BA00000000000000000000000000000000000E5
:106BB00000000000000000000000000000000000D5
:106BC00000000000000000000000000000000000C5
:106BD00000000000000000000000000000000000B5
:106BE00000000000000000000000000000000000A5
:106BF0000000000000000000000000000000000095
:106C00000000000000000000000000000000000084
:106C10000000000000000000000000000000000074
:106C20000000000000000000000000000000000064
:106C30000000000000000000000000000000000054
:106C40000000000000000000000000000000000044
:0C6C500000000000000000000000000038
:086C5C001895FF7F0100000004
:106C6400FFFFFFFF18000000030000000200000007
:106C7400080000000A000000FFFFFFFF0000000002
:106C8400010000000000020001000000FFFFFFFF00
:106C940000000000020000000000040002000000E8
:106CA400FFFFFFFF000000000300000000000800D9
:106CB4000300000000000000F86B0000186C0000E6
:106CC400386C00000000000000000000000000001C
:106CD40000000000BC6A000000000000000000008A
:106CE40000000000000000000000000000000000A0
:106CF4000000000000000000000000000000000090
:106D0400000000000000000000000000000000007F
:106D14000000000054000020F76A00003901000060
:106D2400A53B0000893E0000E54600000D0100007F
:046D3400000000005B
:0400000300003EA11A
:00000001FF
